:100000000C941E060C94B6280C94E3280C94460617
:100010000C9446060C9446060C9446060C94460630
:100020000C9446060C9446060C9422130C94460637
:100030000C9446060C9446060C9446060C94460610
:100040000C9410290C9446060C94FE2C0C94412D13
:100050000C9446060C9446060C9446060C944606F0
:100060000C9446060C94460604196619451948195D
:100070004B194E1951195419571966196019981AC4
:100080009A1A9A1A981A9A1A9A1A9A1A9A1A9A1AD2
:100090009A1A9A1A9A1A9A1A9A1A9A1A9A1A9A1AC0
:1000A0001E1A9A1A9A1A9A1A9A1A9A1A8F199A1A38
:1000B0009A1A9A1A9A1A9A1A9A1A9A1A9A1A9A1AA0
:1000C0009A1A9A1A9A1A9A1A9A1A9A1A2A1A2A1A70
:1000D0002A1A2A1A2A1A2A1A2A1A2A1A2A1A9A1A90
:1000E0009A1A9A1A9A1A9A1A9A1A8F19291A291A5E
:1000F000291A291A9A1A371A3D1A431A491A4F1AF5
:10010000551A5B1A611A6B1A751A7F1A891AD01957
:1001100092199A1A9A1A9A1A9A1A1E1A9A1A9A1AC4
:100120009A1A9A1A9A1A9A1A9A1A9A1A281A281A13
:10013000281A281A9A1A371A3D1A431A491A4F1AB6
:10014000551A5B1A611A6B1A751A7F1A891AD01917
:1001500092199A1A9A1A9A1A9A1A1E1ACD1ACD1A1E
:10016000CD1ACD1ACD1ACD1ACD1ACD1ACD1ACD1A57
:10017000CD1ACD1ACD1AE41BE41BE41BE41BE41BCF
:10018000E41B121B1C1B261B301B8E1B981BA71B62
:10019000B81B401D551D611D6A1D791D9E1DA71DA3
:1001A000F01DB91D032109210F211621242146210B
:1001B0006421456E746572206D656E752E2E2E005D
:1001C000546F67676C6564206D6963726F50504D42
:1001D00000546F67676C656420696E76657274653C
:1001E000642050504D2100546F67676C6564205443
:1001F00058206D7574696E672100546F67676C6570
:10020000642074656C656D65747279210050726F3D
:10021000746F636F6C206572726F72207769746897
:100220002052580054696D656F7574207768656E4B
:1002300020636F6E6E656374696E6720746F205201
:100240005800507265737320616E79206B65792058
:10025000746F2063616E63656C00436F6E6E6563DF
:1002600074696E6720746F2052582C20706F776508
:100270007220757020746865205258202877697440
:10028000682062696E6420706C7567206966206EF4
:100290006F74207573696E6720616C776179732064
:1002A00062696E642900546F67676C656420276912
:1002B0006D6D656469617465206F75747075742700
:1002C00000546F67676C65642027736C61766520E6
:1002D0006D6F64652700546F67676C6564202761E4
:1002E0006C776179732062696E642700546F676769
:1002F0006C65642050504D206368616E6E656C20A3
:100300006C696D69740053657420525353492069B8
:100310006E6A656374696F6E206368616E6E656C8A
:100320002028303D3D64697361626C652900536526
:10033000742050504D206D696E696D756D20737914
:100340006E630053657420626561636F6E20696E31
:1003500074657276616C0053657420626561636FC9
:100360006E2064656C617900536574206265616319
:100370006F6E206672657175656E637920696E2097
:10038000487A3A20303D64697361626C652C205074
:10039000783D504D52206368616E6E656C20782CFC
:1003A0002046783D465253206368616E6E656C202E
:1003B00078005365742050574D2073746F7020641B
:1003C000656C61792028302064697361626C6564B2
:1003D0002C20312D323535203D3D20302E317320FB
:1003E0002D2035306D696E29005365742050504DB5
:1003F0002073746F702064656C61792028302064EC
:10040000697361626C65642C20312D323535203D75
:100410003D20302E3173202D2035306D696E29003E
:10042000536574206661696C736166652064656CF0
:1004300061792028302064697361626C65642C20C6
:10044000312D323535203D3D20302E3173202D2089
:1004500035306D696E29002A2A2A2A2A2A2A2A2A50
:100460002A2A2A2A2A2A2A2A2A2A2A2A2A2A2A2AEC
:100470002A2A2A2A0052582041636B6564202D20C5
:1004800072657665727420737563636573736675E0
:100490006C21002A2A2A2A2A2A2A2A2A2A2A2A2AAD
:1004A0002A2A2A2A2A2A2A2A2A2A2A2A2A2A2A2AAC
:1004B000002A2A2A2A2A2A2A2A2A2A2A2A2A2A2AC6
:1004C0002A2A2A2A2A2A2A2A2A2A2A2A2A2A00528E
:1004D000582041636B6564202D20757064617465DC
:1004E000207375636365737366756C21002A2A2A0D
:1004F0002A2A2A2A2A2A2A2A2A2A2A2A2A2A2A2A5C
:100500002A2A2A2A2A2A2A2A2A2A0056616C696457
:100510002063686F69636573206172653A205B319F
:100520005D2D5B31365D20286368616E6E656C20E1
:10053000312D31362900536574206F7574707574D0
:1005400020666F7220706F727420005B585D2061AE
:10055000626F7274206368616E67657320616E6498
:10056000206578697420525820636F6E6669670051
:100570005B535D20736176652073657474696E6783
:100580007320746F205258005B525D20726576654F
:1005900072742052582073657474696E6773207486
:1005A0006F2064656661756C747300557365206EA9
:1005B000756D62657273205B312D445D20746F2010
:1005C0006564697420706F727473205B452D515D92
:1005D00020666F722073657474696E677300202DD6
:1005E00020726563656976657220636F6E66696700
:1005F000757261746F722C20727820737720000AF4
:100600000A6F70656E4C52536E67200053657420FC
:1006100073657269616C2062617564726174653AB8
:10062000200056616C69642063686F696365733A82
:100630002031202D20342B34202F2032202D203823
:10064000202F2033202D20382B34202F2034202D14
:10065000203132202F2035202D2031322B34202FF5
:100660002036202D20313600536574204368616E9A
:100670006E656C20636F6E6669673A20005365741F
:100680002044617461726174652028302D32293AEA
:10069000200053657420486F70206368616E6E653A
:1006A0006C7320286D61782032342C207365706162
:1006B000726174656420627920636F6D6D61732966
:1006C0002076616C69642076616C75657320312DCC
:1006D0003235353A2000536574206368616E6E656B
:1006E0006C2073706163696E6720287831306B48C5
:1006F0007A293A200053657420524620706F77653E
:10070000722028302D37293A200053657420524634
:10071000206D6167696320286865782920652E67E8
:100720002E20307844454144463030443A2000532E
:1007300065742062617365206672657175656E63AC
:10074000792028696E20487A293A20005B5A5D207A
:10075000656E746572207265636569766572206383
:100760006F6E66696775726174696F6E2075746902
:100770006C79005B465D20646973706C61792061FF
:10078000637475616C206672657175656E63696509
:10079000732075736564005B525D2063616C6375E3
:1007A0006C6174652072616E646F6D206B65792079
:1007B000616E6420686F70206C697374005B495DC2
:1007C000207265696E697469616C697A6520736508
:1007D0007474696E677320746F20736B65746368DB
:1007E0002064656661756C7473005B585D2072658A
:1007F00076657274206368616E67657320616E64EC
:100800002065786974206D656E75005B535D20739B
:100810006176652073657474696E677320746F20E8
:10082000454550524F4D20616E64206578697420B3
:100830006D656E7500557365206E756D62657273BA
:10084000205B302D395D20746F20656469742070E1
:100850006172616D657465727300202D2053797328
:1008600074656D20636F6E66696775726174696F18
:100870006E000A0A6F70656E4C52536E672000510D
:1008800029204F7574707574206265666F726520DB
:100890006C696E6B20283D465329203A2000502970
:1008A00020536C617665206D6F64652028657870D3
:1008B0006572696D656E74616C293A20004F29205C
:1008C00054696D65642042494E44206174207374FC
:1008D000617274757020203A20004E292050504DCE
:1008E000206F7574707574206C696D69746564200F
:1008F000202020203A200044495341424C454400E6
:100900004D292050504D205253534920746F20637D
:1009100068616E6E656C202020203A20004C2920F2
:1009200050504D206D696E696D756D2073796E63E1
:10093000202875732920203A200044495341424C15
:100940004544004B29204661696C736166652062ED
:100950006561636F6E20696E74762E2028312D32AA
:10096000353573293A20004A29204661696C736144
:10097000666520626561636F6E2064656C617920D5
:1009800028302D323535203D3E20313073202D204A
:100990003135306D696E293A200049292046616958
:1009A0006C7361666520626561636F6E206672714B
:1009B0002E203A200048292050574D2073746F7024
:1009C0002064656C6179202020202020203A2000BE
:1009D00047292050504D2073746F702064656C61FE
:1009E00079202020202020203A200046292046611E
:1009F000696C736166652064656C617920202020D4
:100A00002020203A200050574D206368616E6E65AB
:100A10006C200066756E6374696F6E3A2000292041
:100A2000706F72742000506F776572546F776572C3
:100A300000445446205548462033322D62697420C4
:100A400031306368004F70656E4C52536E67525878
:100A5000206D696E6920342F36636800466C7974A6
:100A6000726F6E2F4F72616E6765525820554846FF
:100A70002038636800525820747970653A20004429
:100A8000697361626C656400487A00203D3D200016
:100A900043616C63756C61746564207061636B6540
:100AA0007420696E74657276616C3A200042292068
:100AB0004D6963726F202868616C66292050504D23
:100AC000202020203A00412920496E766572746505
:100AD000642050504D20696E20202020203A0030A4
:100AE00029204D7574652062757A7A657220286DAB
:100AF0006F73746C79293A003929205365726961E2
:100B00006C2062617564726174653A00736D617224
:100B100074506F7274004672536B79005472616E38
:100B200073706172656E740044697361626C6564B0
:100B30000038292054656C656D657472793A2020FF
:100B40002020202020003729204368616E6E656CCC
:100B500020636F6E6669673A202000362920446161
:100B60007461726174652028302D32293A2020206A
:100B700000352920486F70206368616E6E656C7364
:100B80003A2020202020003429204368616E6E65C1
:100B90006C2073706163696E673A202000332920EE
:100BA000524620706F7765722028302D37293A2001
:100BB0002020003229205246206D616769633A2067
:100BC0002020202020202020003129204261736530
:100BD000206672657175656E63793A202020000089
:100BE00000000700020100000304060000000000EE
:100BF00000000001020408102040800102040810D7
:100C00002001020408102004040404040404040263
:100C10000202020202030303030303000000002395
:100C2000002600290000000000250028002B0000FD
:100C3000000000240027002A00002F2E11241FBED0
:100C4000CFEFD8E0DEBFCDBF13E0A0E0B1E0ECE62F
:100C5000F2E602C005900D92A83CB107D9F716E064
:100C6000A8ECB3E001C01D92AE38B107E1F71CE07B
:100C7000CCE3DCE004C02297FE010E94382FCA3387
:100C8000D107C9F70E946B2E0C9434310C940000EC
:100C900080917305813019F482E08093730580910F
:100CA0007305833019F484E0809373050895A89543
:100CB0000895DC01ED91FC910190F081E02D099502
:100CC00008952091740530917505382748E0C901D1
:100CD000880F991F37FF06C09C0151E2252750E17C
:100CE000352701C09C01415091F730937505209341
:100CF0007405089588E38093760580E092ECA1E086
:100D0000B0E08093770590937805A0937905B09330
:100D10007A0587E08093830580EC9AECA9E8B6E336
:100D200080937B0590937C05A0937D05B0937E0511
:100D300085E0809384058DEE9EEFADEABEED809355
:100D40007F0590938005A0938105B0938205E5E827
:100D5000F5E080E090E0863028F4DC01AE54BC4F32
:100D60002C9101C020E0219301968831910599F7DB
:100D700082E080939D058AE080939E05089580EC33
:100D800097EFAAEBB7E38093BB059093BC05A093C4
:100D9000BD05B093BE0580E090E0A0E0B0E5809393
:100DA000BF059093C005A093C105B093C205E3ECC5
:100DB000F5E080E081938F5F8031E1F70895A0E056
:100DC000B0E0E5EEF6E00C94012FD82F0E946629E2
:100DD0006115710581059105C9F30E94A42F109238
:100DE0007F05109280051092810510928205C4E063
:100DF000812C912C54018A94C0907F05D09080055D
:100E0000E0908105F0908205FE2CED2CDC2CCC24AA
:100E10000E949F2FA50194010E94E02E6C0D7D1D64
:100E20008E1D9F1D60937F057093800580938105C3
:100E300090938205C15001F7DD2309F450C005E805
:100E400015E0E801A12CB12C62E3C62ED12CE12CD7
:100E5000F12C8881882309F442C0B39419F40E94CC
:100E60007A063DC00E949F2FA70196010E94E02EA6
:100E7000E1E0E60FA5E8B5E08A2F801B8A1520F493
:100E80008D918E13F9CFE9CF2091840530E0A0E158
:100E9000B7E20E94782E9B01AC01AE2FB0E00E9419
:100EA000872E40907B0550907C0560907D0570906A
:100EB0007E05640D751D861D971D4090BB055090E5
:100EC000BC056090BD057090BE05461657066806C5
:100ED000790618F2E993A39488E1A812BACFCDB7A6
:100EE000DEB7E0E10C941D2F8436910520F4BC019F
:100EF00080E090E017C09C018E3B910528F42A55B4
:100F00003109AAE0B0E00CC0823D910528F4245BD1
:100F10003109A4E6B0E004C02D5C3109A8E5B2E0D7
:100F20000E94782EA4E6B0E09B01AC010E94872EBF
:100F3000089590E08C599F4F0E947407089561E0D6
:100F400086E00E94132A60E086E00E944C2A82E03C
:100F50008093B00085E08093B10061E083E00E945F
:100F6000132A60E083E00E944C2A0895CF93DF9318
:100F7000EC010097E9F061E086E00E944C2A9E01B6
:100F800040E050E068E478EE81E090E00E94E02EDE
:100F90002F3F31054105510529F020F02FEF30E0BA
:100FA00040E050E02093B3008091B000806107C022
:100FB00060E086E00E944C2A8091B0008F7E809392
:100FC000B000DF91CF91089560E08EE00E94132A77
:100FD00061E08FE00E94132A61E080E10E94132A01
:100FE00060E082E00E94132A61E084E00E94132AFC
:100FF000089542E050E068E476E080E00E949628A0
:101000000895E3E0F0E089E080935700E491E67012
:1010100081E0E63009F080E00895CF93DF93C82F98
:101020000E940108882381F0DFB781E08093720578
:10103000F8940E94570688E180936000C093600096
:10104000C1110E945706DFBFDF91CF9108958F92A3
:101050009F92AF92BF92CF92DF92EF92FF92CF9387
:10106000FC01C0A5EC2FE770F0E0E658FC4FA08132
:10107000B0E0C7FF03C024E130E002C02FE030E061
:10108000FC0197A183E1989FF0011124E25CFE4FDF
:1010900080809180A280B380A20FB31F20E43FE143
:1010A0004DE750E00E94922EA50194010E94BE2EB1
:1010B0008C2F887149F469017A01E0EDCE0EE7E0EA
:1010C000DE1EE11CF11C1BC0C7FF05C060E47AE80E
:1010D0008CE29EE004C060E07EEE8AEB9BE069015A
:1010E0007A01F8EBCF0EFBE0DF1EE11CF11CA5013D
:1010F00094010E94BE2EC20ED31EE41EF51EC7012F
:10110000B60169517C4F8F4F9F4F28EE33E040E08E
:1011100050E00E94BE2EA8EEB3E00E94872ECF9131
:10112000FF90EF90DF90CF90BF90AF909F908F9007
:1011300008958F3F910551F048F0811522E0920704
:1011400038F08115934030F482E0089580E00895EE
:1011500081E0089583E00895A0E0B0E0E2EBF8E0DC
:101160000C940A2FEB018A01B82FB695A0E02881D4
:101170003981F80120832A813B8121832C813D81A3
:1011800022832E813F812383688179814A815B811B
:101190002C813D81EE81FF819F2F9295990F990FB0
:1011A000907C272F2370922B252F2370220F220F44
:1011B000922B232F23702295207F922BF80194836A
:1011C0000B5F1F4F2896AF5FBA1788F680FF24C0C9
:1011D000888199810E949908D82E8A819B810E94DA
:1011E0009908E82E8C819D810E949908F82E8E81A5
:1011F0009F810E949908F0E4DF9EA001112490E1F4
:10120000E99E90011124242B282BE4E0FE9EB001DE
:101210001124262BF8012083CDB7DEB7E7E00C942C
:10122000262F803223E0920708F1883E23E09207C0
:1012300040F48F519340E4E096958795EA95E1F765
:101240000895803D27E0920718F48C5D934008953F
:10125000883928E0920768F4885C974074E0969596
:1012600087957A95E1F78D509C4F089580E090E046
:1012700008958FEF93E008958C30910540F4A4E039
:10128000880F991FAA95E1F7885D9C4F0895843FC8
:1012900023E0920718F484529C4F0895811524E0AE
:1012A000920740F48657934FF4E0880F991FFA9500
:1012B000E1F7089580E998E008959C013695279517
:1012C00025753575821B930B9C012373337396959B
:1012D00087959695879583739373820F931F9C01CF
:1012E00054E0369527955A95E1F7280F391F2F704E
:1012F0003F7041E051E0249FC001259F900D349F35
:10130000900D1124892F08954298882319F0000028
:10131000419A02C0000041980000429A00000895DE
:10132000429A000086B14298000081700895CF93E0
:10133000DF93D82F5C9A42985C98C8E08D2F807814
:101340000E948409DD0FC150C9F74298DF91CF9107
:1013500008958F770E9497090895CF93DF93D82F30
:10136000C8E08D2F80780E948409DD0FC150C9F735
:101370004298DF91CF910895CF93DF934298C8E0D0
:1013800080E0D82FDD0F0E9490098D0FC150C9F762
:10139000DF91CF9108950E94A9090E94BC095C9A2F
:1013A0000895A1E0B0E0E7EDF9E00C940F2F80681C
:1013B00069830E9497096981862F0E94AD095C9A12
:1013C0002196E2E00C942B2FCF93C0917F05C82784
:1013D000E82FF0E0EA58FA4F678589E70E94D109C3
:1013E0006C2F8DE30E94D1096C2F82E40E94D109F9
:1013F000CF91089586E20E94CB090895CF93DF93A1
:10140000EC016C818CE10E94D1096D818DE10E941B
:10141000D1096E818EE10E94D1096F8180E20E9424
:10142000D109688581E20E94D109698582E20E9422
:10143000D1096A8583E20E94D1096B8584E20E940A
:10144000D1096C8585E20E94D1096D858AE20E94EE
:10145000D1096E858EE60E94D1096F858FE60E94C4
:10146000D109688980E70E94D109698981E70E94D2
:10147000D1096A8982E70E94D109DF91CF9108954D
:10148000CF92DF92EF92FF92CF93DF936B017C01BB
:10149000C11488E3D8068CE9E8068CE1F80628F543
:1014A000C701B60120E836E948E950E00E94BE2EA7
:1014B000E901689760E879E687E69FEF0E949A2E37
:1014C0006C0D7D1D8E1D9F1DF2E0660F771F881F1E
:1014D000991FFA95D1F721E732E040E050E00E94F1
:1014E000BE2EF22EE32E80E421C0C701B60120E01B
:1014F0003DE241E351E00E94BE2EE901689760E0C1
:1015000073ED8EEC9EEF0E949A2E6C0D7D1D8E1D4C
:101510009F1D660F771F881F991F21E732E040E06B
:1015200050E00E94BE2EF22EE32E80E66C2F6F71EB
:10153000680F85E70E94D1096E2D86E70E94D109C8
:101540006F2D87E70E94D109DF91CF91FF90EF9037
:10155000DF90CF900895682F8DE60E94D1090895FD
:101560008F929F92AF92BF92CF92DF92EF92FF92B3
:10157000CF93DF93D82F83E00E94CB09809371052E
:1015800084E00E94CB098093700560E086E00E94B1
:10159000D10961E087E00E94D1096FE789E00E94EC
:1015A000D10965E08AE00E94D10962E18BE00E94E6
:1015B000D10965E18CE00E94D1096DEF8DE00E94B8
:1015C000D10960E08EE00E94D109DD2319F08BE2A1
:1015D00091E008C020919D0533E1239FC0011124B3
:1015E000825C9E4F0E94FE096CE880E30E94D10954
:1015F0006FE082E30E94D10962E483E30E94D10993
:1016000080919E0587FF02C064E101C06AE084E327
:101610000E94D1096AE285E30E94D1096DE286E366
:101620000E94D10964ED87E30E94D10960E088E35C
:101630000E94D10960E089E30E94D109D11109C05B
:10164000C0907F05D0908005E0908105F0908205E4
:1016500007C0C5E9CC2EC1ECDC2EED2CCEEDFC2E66
:10166000CAE38F2C9924AA24BB24682D8C2F0E94B6
:10167000D109682D85E08C0F0E94D109FE2CED2C3C
:10168000DC2CCC24CF5FCE3361F76FEF83E40E9474
:10169000D1096FEF84E40E94D1096FEF85E40E94C5
:1016A000D1096FEF86E40E94D109DD2311F066E0D5
:1016B00002C0609183058DE60E94D10960E089E750
:1016C0000E94D109609184058AE70E94D10960E0F7
:1016D00083E70E94D10960E084E70E94D109D1111B
:1016E00009C060917B0570917C0580917D0590918A
:1016F0007E0504C060EC7AEC89E896E30E94400A1B
:10170000DF91CF91FF90EF90DF90CF90BF90AF909F
:101710009F908F90089561E087E00E94D10964E274
:101720008EE70E94D10963E088E00E94D10960E061
:1017300088E00E94D10965E087E00E94D10962E05B
:1017400085E00E94D10983E00E94CB098093710556
:1017500084E00E94CB0980937005089583E00E9485
:10176000CB098093710584E00E94CB0980937005BA
:1017700061E087E00E94D1096AE070E080E090E0DB
:101780000E9489290E948B0B00000895CF92DF925E
:10179000FF920F931F93CF93DF931F92CDB7DEB7C6
:1017A000082F162F8EE399830E94D109F02EC02EA8
:1017B0009981D92E8C2D8F19811738F4F6016191FA
:1017C0006F018FE70E94D109F5CF64E085E00E94A8
:1017D000D10983E00E94CB098093710584E00E94C7
:1017E000CB09809370050E94662960936C05709305
:1017F0006D0580936E0590936F0569E087E00E9408
:10180000D10981E0809373050F90DF91CF911F91F3
:101810000F91FF90DF90CF9008950F931F930E9438
:10182000C60B80917305813099F40E94662900915E
:101830006C0510916D0520916E0530916F05601B50
:10184000710B820B930B603A76488140910548F307
:1018500080917305813031F46EE971E082EE95E09C
:101860000E94522B1F910F9108950F931F93809107
:101870007305823021F41092730581E020C08091BD
:1018800073058130D9F40E94662900916C0510918E
:101890006D0520916E0530916F05601B710B820BF9
:1018A000930B613A76488140910540F061E087E012
:1018B0000E94D1091092730582E001C080E01F915F
:1018C0000F910895CF93DF93EC014AE050E06D2F24
:1018D00070E082EE95E00E94202C6EE282EE95E0B0
:1018E0000E94242BBE0184E0769567958A95E1F7E6
:1018F0006F7077274AE050E082EE95E00E94202C3E
:101900006EE282EE95E00E94242BBE016F70772775
:101910004AE050E082EE95E00E94202CDF91CF91CA
:101920000895D82FC0E0CD1790F4439A299A64E621
:1019300070E080E090E00E9489294398299864E64D
:1019400070E080E090E00E948929CF5FECCF6CE2EC
:1019500071E080E090E00E948929E4CF0F931F930B
:10196000CF93DF93EC01062F15E0115051F0CE011B
:101970000E941B31081741F0602FCE010E942331D5
:10198000F4CF82E00E94910CDF91CF911F910F91D3
:101990000895A0E0B0E0EFECFCE00C94012F482E9D
:1019A000562EC0E0D0E0612C712CE12CF12C00E02F
:1019B00010E041100CC06090D40586E4689E3001B0
:1019C000112459E1E52EF12C0AEB15E01EC091E03F
:1019D00049120FC06090D405E6E46E9E30011124D8
:1019E000FBE16F0E711C49E2E42EF12C06E715E0D5
:1019F0000CC082E0481209C028E1622E772473945B
:101A0000EE24E394F12C03ED15E043018C0E9D1EB2
:101A100010927505109274053401A62CA818B12CEB
:101A2000C30101966C01AE14BF04A8F4A00EB11E50
:101A3000511006C0C3010E941B31F501808305C00F
:101A4000F5016081C3010E94AE0CF50180810E9406
:101A500061063601E2CFC301511018C0C3010E94D4
:101A60001B31B82EC6010E941B312B2D30E0322FC6
:101A70002227282B80917405909175058217930772
:101A800079F4C0E0D0E05524539493CF36016091AF
:101A900075050E94AE0C60917405C6010E94AE0CE3
:101AA000C05EDE4FC13E92E0D90708F482CF852D9B
:101AB000CDB7DEB7E0E10C941D2F61E082E00E941B
:101AC000C90C089560E082E00E94C90C8091D305A2
:101AD000853020F01092D3050E945D0D8091D305D2
:101AE0008093D405089561E080E00E94C90C61E014
:101AF00081E00E94C90C089560E080E00E94C90C5A
:101B0000882351F060E081E00E94C90C882321F015
:101B100080917605883349F00E94BF060E947A06BC
:101B200081E00E94DF060E94730D0895882319F05A
:101B30006AEA71E002C06EEA71E082EE95E00E940E
:101B4000522B0895FF920F931F93CF93DF9369EC6D
:101B50007BE082EE95E00E94FE2A40917B05509149
:101B60007C0560917D0570917E052AE030E082EE73
:101B700095E00E94272C63EB7BE082EE95E00E94CB
:101B8000FE2A40917F0550918005609181057091FA
:101B9000820520E130E082EE95E00E94272C6DE97D
:101BA0007BE082EE95E00E94FE2A4AE050E06091E0
:101BB000830582EE95E00E944F2C67E87BE082EE81
:101BC00095E00E94FE2A4AE050E06091840582EE92
:101BD00095E00E944F2C61E77BE082EE95E00E9449
:101BE000FE2AC5E8D5E0F12C8E0188818823A9F072
:101BF000FF2031F061EB71E082EE95E00E94212B35
:101C000021964AE050E0F801608182EE95E00E9462
:101C1000182CF394F8E1FF12E7CF82EE95E00E94D2
:101C20002C2B6BE57BE082EE95E00E94FE2A4AE0D9
:101C300050E060919D0582EE95E00E944F2C66E495
:101C40007BE082EE95E00E94FE2AE0919E05E7701F
:101C5000F0E0EE0FFF1FEE57FC4F6081718182EEC6
:101C600095E00E94522B61E37BE082EE95E00E94BA
:101C7000FE2A80919E058871883069F028F48111D0
:101C800013C068E27BE00CC0803141F0883161F420
:101C90006CE07BE005C06CE17BE002C066E17BE0CC
:101CA00082EE95E00E94402B68EF7AE082EE95E0AC
:101CB0000E94FE2A40917705509178056091790540
:101CC00070917A052AE030E082EE95E00E94272CA0
:101CD0006FED7AE082EE95E00E94FE2A8091BF05CA
:101CE00080710E94960D66EC7AE082EE95E00E948B
:101CF000FE2A8091BF0580740E94960D6DEA7AE0FD
:101D000082EE95E00E94FE2A8091BF0580720E94BB
:101D1000960D60E97AE082EE95E00E94FE2A86E761
:101D200095E00E942708AB01BC012AE030E082EE7A
:101D300095E00E94092C6BE87AE082EE95E00E9423
:101D4000FE2A86E795E00E9427089B01AC0160E42B
:101D500072E48FE090E00E94BE2EBA01A9012AE051
:101D600030E082EE95E00E94092C68E87AE082EE8D
:101D700095E00E94402BCDB7DEB7E5E00C94282F0C
:101D80008F929F92AF92BF92CF92DF92EF92FF928B
:101D9000811107C06FE77AE082EE95E00E94402B48
:101DA0002FC090E00E94740724E630E040E050E04D
:101DB0000E94BE2ECA01B9012AE030E040E050E0A6
:101DC0000E94BE2E49015A016B017C012AE030E0DD
:101DD000B501A40182EE95E00E94092C6EE282EE2C
:101DE00095E00E94242B2AE030E0B701A60182EEA4
:101DF00095E00E94092C63E782EE95E00E94642B37
:101E0000FF90EF90DF90CF90BF90AF909F908F901A
:101E100008951F93CF93DF9365E77AE082EE95E014
:101E20000E94FE2A80919F05813041F46CE57AE0A2
:101E300082EE95E00E94402B10E050C0823019F4F1
:101E400065E47AE0F5CF843019F461E37AE0F0CF0D
:101E5000853091F766E27AE0EBCFC12FD0E0C93050
:101E6000D1050CF441C068E3610F82EE95E00E9459
:101E7000242B6EE17AE082EE95E00E94FE2ABE01FC
:101E80006F5F7F4F4AE050E082EE95E00E94E82BC2
:101E900063E17AE082EE95E00E94FE2AC156DA4FB5
:101EA000E981E03218F566E07AE082EE95E00E9482
:101EB000FE2A8981803130F06DE673E082EE95E094
:101EC0000E94212B69816F7070E06F5F7F4F4AE045
:101ED00050E082EE95E00E94F12B1F5F8091480553
:101EE000181708F4BACF0FC061E3BECFEF70F0E06F
:101EF000EE0FFF1FEE56FC4F6081718182EE95E080
:101F00000E94522BEACF6BEE79E082EE95E00E94C0
:101F1000FE2A8091B7050E94C00E60ED79E082EE46
:101F200095E00E94FE2A8091B8050E94C00E65EBE4
:101F300079E082EE95E00E94FE2A8091B9050E9428
:101F4000C00E6AE979E082EE95E00E94FE2A409197
:101F5000AF055091B0056091B1057091B205411582
:101F600051056105710539F12AE030E082EE95E016
:101F70000E94272C67E679E082EE95E00E94FE2A17
:101F80008091B3050E949907AB01BC012AE030E0C3
:101F900082EE95E00E94272C63E479E082EE95E0E2
:101FA0000E94FE2A4AE050E06091B40582EE95E07E
:101FB0000E944F2C06C06AE379E082EE95E00E9411
:101FC000402B6DE179E082EE95E00E94FE2A60915F
:101FD000B5057091B6054AE050E082EE95E00E94AA
:101FE000392C60E079E082EE95E00E94FE2A609153
:101FF000AE05603450F470E06F5F7F4F4AE050E010
:1020000082EE95E00E94F12B06C067EF78E082EE49
:1020100095E00E94402B6AED78E082EE95E00E9408
:10202000FE2A8091AD0580FF03C063EB71E002C022
:1020300067EB71E082EE95E00E94522B6DEB78E049
:1020400082EE95E00E94FE2A8091AD0582700E948A
:10205000960D6EE978E082EE95E00E94FE2A80916E
:10206000AD0584700E94960D6FE778E082EE95E0F2
:102070000E94FE2A8091AD0588700E94960DDF9126
:10208000CF911F9108950F931F93CF93DF932091CA
:1020900045052F3FA9F56FEF75E082EE95E00E94B0
:1020A000FE2A84E893E00E94620C6EED75E082EEF9
:1020B00095E00E94FE2A80914605909147050E9476
:1020C000620C6BEA75E082EE95E00E94402B68E8B6
:1020D00075E082EE95E00E94402B60E775E082EEAD
:1020E00095E00E94402B6BE475E082EE95E00E9443
:1020F000402B82EE95E00E942C2B0E94090F68C0B5
:1021000012160CF065C0332727FD309580914805E5
:1021100090E0821793070CF45BC066E375E082EEF3
:1021200095E00E94FE2A60914505772767FD70952E
:102130004AE050E082EE95E00E94F12B6BE075E002
:1021400082EE95E00E94FE2A10E008E280914905A7
:102150001817D0F5C12FD0E0CC0FDD1FC65BDA4FCA
:10216000288130E080914505992787FD909501975A
:102170002817390739F56BEB71E082EE95E00E9484
:10218000212B4AE050E0602F82EE95E00E94182C4F
:102190006FEB71E082EE95E00E94212BE981EF70F8
:1021A000F0E0EE0FFF1FEE56FC4F6081718182EE72
:1021B00095E00E94212B63EC71E082EE95E00E9495
:1021C000212B0F5F1F5FC2CF82EE95E00E942C2B68
:1021D000DF91CF911F910F910895FF920F931F935D
:1021E000CF93DF93C5E8D5E0F12C8E018881882359
:1021F000D1F165EC71E082EE95E00E94212B4AE07E
:1022000050E06F2D82EE95E00E94182C62ED71E097
:1022100082EE95E00E94212B2196F801208130E08A
:10222000A0E1B7E20E94782E9B01AC01A091840549
:10223000B0E00E94872EAB01BC0180917B0590919C
:102240007C05A0917D05B0917E05480F591F6A1F3E
:102250007B1F2AE030E082EE95E00E94272CF39469
:10226000F8E1FF12C2CFCDB7DEB7E5E00C94282F1E
:102270001092DF0485E6E0EEF4E0DF011D928A951E
:10228000E9F70895CF93C82F8F3719F0883009F0F8
:1022900045C0E091DF04EE23D9F1E150E093DF0483
:1022A000F0E0E052FB4F10826DE070E082EE95E0CE
:1022B0000E945906C0E08091DF04C81760F4EC2F3B
:1022C000F0E0E052FB4F608170E082EE95E00E940A
:1022D0005906CF5FF0CF60E270E082EE95E00E9499
:1022E00059066DE070E082EE95E00E945906C0E06C
:1022F0008091DF04C81778F5EC2FF0E0E052FB4F37
:10230000608170E082EE95E00E945906CF5FF0CFC9
:1023100067E082EE95E00E94242B1DC08B3119F4FA
:102320000E9438111AC08D30C1F08A30B1F080910E
:10233000DF04843668F76C2F70E082EE95E00E942F
:102340005906E091DF0481E08E0F8093DF04F0E016
:10235000E052FB4FC08380E001C081E0CF9108953F
:10236000CF93C82F0E9466296093C8047093C90454
:102370008093CA049093CB04C093DD04CC2329F04E
:1023800040E051EE60E070E004C040E855E260E0FB
:1023900070E082EE95E00E94AE2DCF91089590916D
:1023A000CC04492F4F7050E0BA016F5F7F4F292F47
:1023B00030E0E4E035952795EA95E1F76217730779
:1023C00059F0FA01E353FB4F808381E0890F8F704E
:1023D000907F892B8093CC0408956EE770E082EEA5
:1023E00095E00E9459060895A3E1B1E0EAEFF1E11A
:1023F0000C94022FE5E8F5E0712C8191882321F0FF
:10240000739428E17212F9CF66ED71E082EE95E0E7
:102410000E94522B4AE050E0672D82EE95E00E9428
:102420004F2C80E00E94B00A0E948B0B8E010E5F41
:102430001F4FC12CD12C7601C39466246A945C2C66
:102440000E945A294B015C012091840530E0A0E1F3
:10245000B7E20E94782E9B01AC01C701B6010E9431
:102460009A2E20917B0530917C0540917D055091FD
:102470007E05620F731F841F951F2091BB0530914D
:10248000BC054091BD055091BE052617370748078A
:10249000590718F4F80160822AC08C2D0E94E409C3
:1024A00061E070E080E090E00E948929F8011082EC
:1024B0000E945A29681979098A099B09643F714069
:1024C0008105910540F40E94FA09F801908198175E
:1024D00078F78083EDCF85B150FE05C08B7D85B93F
:1024E000439A299A04C0846285B9439829982FEFAA
:1024F000C21AD20AE20AF20A0F5F1F4F8FEFC81604
:10250000D104E104F10409F09ACFCE019395FC01C6
:10251000D82E7FEF68EC2E2F281B271510F051E0E6
:1025200056C0DE01129651E02FEF41E03D91321787
:1025300010F0322F01C0452F5F5F5F3F11F0232F56
:10254000F5CF4193242F30E0A1E0B0E0AC0FBD1FE8
:10255000A20FB31F5C93413079F0DE01A20FB31FCD
:102560005C93423049F0AFEFBFEFAC0FBD1FA20F3D
:10257000B31F6C934E3F78F6A2E0B0E0AC0FBD1FE6
:10258000A20FB31F7C934D3F30F6A3E0B0E0AC0F39
:10259000BD1FA20FB31F6C93BECF452F242F30E079
:1025A000FC01E20FF31F6081AFEFB0E0AC0FBD1F85
:1025B000A20FB31F2C91621748F44150DC01A40F05
:1025C000B11D2C9120836C934111E8CF5F5F5715AB
:1025D00020F3372D369520E0231770F4DC01A20F8D
:1025E000B11D4C91522F530FFC01E50FF11D50818D
:1025F0005C9340832E5FF0CFF5E8EF2EF5E0FF2EE1
:102600008C01802F8D19871598F4F801C1908F01E6
:102610004AE050E06C2D82EE95E00E94182C6CE2AE
:1026200082EE95E00E94242BF701C1927F01E9CF51
:1026300082EE95E00E942C2B81E0CD5EDE4FEFE034
:102640000C941E2F1F920F920FB60F9211241F93FE
:102650002F933F934F935F936F937F938F939F93AA
:10266000AF93BF93CF93DF93EF93FF93C091860017
:10267000D091870080918704909188042091A904CB
:10268000211155C09E01281B390B8091BF059091E7
:10269000C005A091C105B091C20585FD02C0369567
:1026A0002795253C49E03407B8F140910A0150E0F4
:1026B00060E070E02CE1B695A795979587952A95EF
:1026C000D1F70097A105B10521F481E090E0A0E0E9
:1026D000B0E084179507A607B707D8F480910A01E0
:1026E0008F3FB9F040E080910A01481780F4842FB1
:1026F00090E0880F991FFC01E757FB4F2081318143
:10270000FC01E55FFE4F318320834F5FECCF1092D9
:10271000AA0410920A010BC02D3B82E0380720F07A
:1027200080910A018031D8F08FEF80930A01D09315
:102730008804C0938704FF91EF91DF91CF91BF91FF
:10274000AF919F918F917F916F915F914F913F9149
:102750002F911F910F900FBE0F901F901895109101
:102760000A0181E0810F80930A01C9010E941109C9
:10277000E12FF0E0EE0FFF1FE757FB4F91838083BF
:10278000D6CF83E0809380008AE980938100809196
:10279000BF0586FD05C08091810080648093810023
:1027A0008FEF9FEF909389008093880080916F0056
:1027B000806280936F000895CF93DF930E94620D33
:1027C0008091D405843039F58BE00E947F2AC1E0E6
:1027D000D0E0892B11F4C0E0D0E08CE00E947F2A89
:1027E000892B19F082E090E002C080E090E08C2B11
:1027F0009D2B8230910539F08330910539F0019796
:1028000039F481E006C01092D40505C082E001C011
:1028100083E08093D405DF91CF9108956F3018F055
:1028200086958058089589E0689F802D1124089529
:10283000A0E0B0E0EEE1F4E10C94092FC82F0E9473
:102840006629009138041091390420913A0430919E
:102850003B046B017C01C01AD10AE20AF30A97011A
:10286000860149E8C41643E1D406E104F10410F0FE
:1028700010923C04609338047093390480933A04B6
:1028800090933B042091A9048FEF820F8230D8F5FA
:10289000E0913C04EE2309F44EC1E13011F482E0F2
:1028A000B8C1E03108F034C181E08E0F80933C0460
:1028B000F0E0E757FB4FC083803109F0ACC1EBE893
:1028C000F4E0213029F4A181A695A695808108C065
:1028D00080819181A92FA695A695A6959695879515
:1028E000A03148F4B0E090E0AA0FBB1FA55FBE4F37
:1028F00011969C938E931092AA04329684E0E93943
:10290000F807F9F688C1233009F005C1E0913C04CD
:10291000E11104C0CF3009F07EC10DC1E83148F4A7
:1029200081E08E0F80933C04F0E0E857FB4FC083BA
:1029300072C1E83109F0ECC0C111EAC040E050E0DA
:10294000ABE0CA01B3E0880F991FBA95E1F7A49FE5
:102950009001A59F300D1124F901E757FB4F6081CD
:10296000E1817E2F777075956795FC01EE0FFF1F53
:10297000E55FFE4F71836083F901E657FB4FB0813D
:10298000B695B695B695E181FE2FF295FF0FF07ED4
:102990006F2F6B2BE695E695E6957E2F77707595F4
:1029A0006795FC01EE0FFF1FE35FFE4F71836083AD
:1029B000F901E557FB4FB081B295B695B695B37066
:1029C000C181DC2FDD0FDD0F6D2F6B2BC295C695FE
:1029D000C695C370E281E170EE0FEE0F7E2F7C2B67
:1029E00075956795FC01EE0FFF1FE15FFE4F718348
:1029F0006083F901E357FB4FB081B695E181FE2F6B
:102A0000F795FF27F7956F2F6B2BE6957E2F777045
:102A100075956795FC01EE0FFF1FEF5EFE4F71830A
:102A20006083F901E257FB4FB081B295BF70E1813D
:102A3000FE2FF295F07F6F2F6B2BE295EF707E2FBC
:102A4000777075956795FC01EE0FFF1FED5EFE4FE9
:102A500071836083F901E157FB4FB081BB1FBB2736
:102A6000BB1FC181DC2FDD0F6D2F6B2BCC1FCC2743
:102A7000CC1FE281E370EE0F7E2F7C2B759567955E
:102A8000FC01EE0FFF1FEB5EFE4F71836083F901C7
:102A9000EF56FB4FB081B695B695E181FE2FF295CA
:102AA000FF0FFF0FF07C6F2F6B2BE695E6957E2FC7
:102AB000777075956795FC01EE0FFF1FE95EFE4F7D
:102AC00071836083F901EE56FB4F20812295269594
:102AD00027703181E32FEE0FEE0FEE0F6E2F622B7A
:102AE000732F72957695777075956795FC01EE0F4B
:102AF000FF1FE75EFE4F718360834F5F5F4F423081
:102B0000510509F01ECF80919F0483FF1092AA0403
:102B100010923C0480C0243009F07DC060913C04D8
:102B200061110BC0C83AB1F410927505109274058A
:102B300088EA0E94610681E06CC0613019F4C0939C
:102B4000370404C0623031F4C09336048C2F0E94E5
:102B500061065AC0E09136042E2F30E0220F331F59
:102B6000462F50E0C9010296841795073CF0633266
:102B700068F7FA01EA57FB4FC083E8CF2D5F3F4F5C
:102B80008C2F90E060917405709175054217530782
:102B900049F4982F88278627972790937505809367
:102BA000740532C06817790769F580913704813060
:102BB00049F5E13118F080E180933604F090360455
:102BC000CAE8D4E000E010E00F15D0F4FE01319720
:102BD000808190E0982F88272881822B63E096954A
:102BE00087956A95E1F70E941109F801EE0FFF1F22
:102BF000E55FFE4F918380830F5F1F4F2296E4CFE6
:102C00001092AA0410923C0480913C04882319F08D
:102C10008F5F80933C04CDB7DEB7E8E00C94252F9E
:102C2000CF93DF93E82FF0E0E654FA4FE185E031EF
:102C300050F4F894F0E0EE0FFF1FE55FFE4F808147
:102C4000918178945DC08EE08E0F8B3058F4F0E067
:102C5000E25FF10924E62E9FC0012F9F900D112401
:102C60000C964EC0E03F09F446C038F4E13181F0E3
:102C7000E23191F0E03139F409C0ED3FB1F1EE3FBE
:102C8000B9F1E13F79F180E092E03AC082E101C020
:102C900083E10E94A82A34C08BE00E947F2AC1E011
:102CA000D0E0892B11F4C0E0D0E08CE00E947F2AB4
:102CB000892B19F082E090E002C080E090E08C2B3C
:102CC0009D2B8230910541F08330910541F00197B1
:102CD000A9F086EA92E014C08CE090E011C089E58A
:102CE00091E00EC086E090E00BC08AEF93E008C050
:102CF0008FEF93E005C080E090E002C084EF93E0A6
:102D0000DF91CF910895A2E2B0E0E9E8F6E10C94FA
:102D1000FF2E9E012F5F3F4F80E1D9011D928A95C2
:102D2000E9F764E072E082EE95E029A33AA30E94FD
:102D3000522B0E94AE0B1D8A1E8A1F8A188E312CC0
:102D4000212C00E0812C912C540170EC472E7DE960
:102D5000572E78E5672E75E3772EE0E5CE2EE3EC6F
:102D6000DE2EE12CF12C84EF91E0A0E0B0E08D8F1D
:102D70009E8FAF8FB8A380EC97EFAAEBB7E3898F54
:102D80009A8FAB8FBC8F80EC9DE9A8E5B5E3898B6A
:102D90009A8BAB8BBC8B82EE95E00E94662C892BC4
:102DA00009F4E1C082EE95E00E94932C9C01332748
:102DB0002C32310509F442C0ACF42332310509F05C
:102DC000ABC019821A821B821C821D821E821F8246
:102DD000188619861A861B861C861D861E861F86E7
:102DE000188A60C02434310529F02335310509F4EF
:102DF000B2C092C064E482EE95E00E94242B2AE0E7
:102E000030E040EC5DE968E575E382EE95E00E9414
:102E1000B22B6CE282EE95E00E94242B2AE030E097
:102E200040EC57EF6AEB77E382EE95E00E94B22B1D
:102E30006CE282EE95E00E94642BADCF0F5F043010
:102E400009F0A9CF29813A814B815C81A8EEB3E0DA
:102E50000E94872E698B7A8B8B8B9C8B2D813E8178
:102E60004F8158850E94872E698F7A8F8B8F9C8F18
:102E700029853A854B855C852D8F3E8F4F8F58A3D2
:102E80002D853E854F8558890E94872E6B017C01D8
:102E900060323EE473078105910530F462E38CE112
:102EA0000E94D10900E077CF603345E774078105C0
:102EB000910510F462E2F3CF60345CE97507810597
:102EC000910510F466E2EBCF80E5C81683ECD806D6
:102ED000E104F10410F462E1E2CF90E6C9169AEE43
:102EE000D906E104F10410F465E1D9CFA0E7CA16D0
:102EF000A1E1DA06A1E0EA06F10410F461E0CFCF27
:102F0000B0EACB16B6E8DB06B1E0EB06F10410F44C
:102F100063E0C5CF65E0C3CF10ED180F1A3008F09D
:102F20003ACFE1E0F0E0EC0FFD1F24E0029FE00D5E
:102F3000F11D11242081318142815381AAE0B0E04A
:102F40000E94872E610F711D811D911D6083718309
:102F50008283938320CF49885A886B887C88812C10
:102F6000912C540118CF81149104A104B10489F467
:102F7000C301B2010E94400A61E070E080E090E08D
:102F80000E9489291D8A1E8A1F8A188E312C2224AC
:102F90002A948D8D9E8DAF8DB8A188169906AA06AC
:102FA000BB06D0F40E94FA092D893E894F89588DBD
:102FB000280F311D411D511D2D8B3E8B4F8B588F7E
:102FC000381608F4382E821508F4282E3FEF831A9D
:102FD000930AA30AB30A56C0C301B20128EE33E034
:102FE00040E050E00E94BE2EBA01A9012AE030E084
:102FF00082EE95E00E94092C6CE282EE95E00E9440
:10300000242B4AE050E0632D82EE95E00E94182CBC
:103010006CE282EE95E00E94242B6D897E898F8977
:10302000988DA50194010E94BE2EBA01A9012AE043
:1030300030E082EE95E00E94092C6CE282EE95E091
:103040000E94242B4AE050E0622D82EE95E00E941F
:10305000182C6CE282EE95E00E94642B4C0C5D1CF7
:103060006E1C7F1C898D9A8DAB8DBC8D841595054A
:10307000A605B70520F449885A886B887C88812C7E
:10308000912C540129893A894B895C89283E334027
:103090004105510509F07FCEA296E2E10C941B2F69
:1030A000ACE1B0E0E6E5F8E10C94092F0E94662956
:1030B0006B017C0181E00E94B00A14E703E01983F0
:1030C00061E0CE0101960E940D0C009373050E94F1
:1030D0008B0B6AEF70E080E090E00E94892980917C
:1030E0007305833089F482EE95E00E94662C892B6B
:1030F00059F40E9466296C197D098E099F09603870
:10310000734C894C9140D8F280917305833009F457
:103110004FC08FE70E94A9090E94BC0989838435AA
:1031200011F083E05CC00E94BC09109246058093B8
:1031300047050E94BC092091460530914705280F9C
:10314000311D30934705209346050E94BC098093AA
:1031500048050E94BC0980934905813110F7F12C84
:103160000F2D10E08091490590E0880F991F0817F6
:10317000190740F40E94BC09F801E65BFA4F80830E
:10318000F394EECF80E7898361E0CE0101960E943F
:103190000D0C83E0809373050E948B0B62E370E05B
:1031A00080E090E00E94892980917305833011F4BA
:1031B00082E015C08FE70E94A9090E94BC0989839B
:1031C000803509F0AECF0FE915E00E94BC09F80187
:1031D00081938F01F5E00A3B1F07B9F781E06C96F8
:1031E000E8E00C94252F80914505992787FD90955F
:1031F000A92FB92FFC013196EB30F10508F066C01C
:10320000EC5CFF4F0C94362F62E778E082EE95E09D
:103210000E94402B84E893E00E94620C6AE578E00B
:1032200082EE95E00E94402B65E378E082EE95E027
:103230000E94402B6BE078E082EE95E00E94402BEC
:103240006AEE77E082EE95E00E94402B6DEB77E02E
:1032500082EE95E00E94402B67E977E082EE95E0F0
:103260000E94402B63E777E082EE95E00E94402BBE
:103270006CE477E082EE95E00E94402B82EE95E0D0
:103280000E942C2B0E94A20D21C06FE277E01AC091
:103290006AE077E017C065EF76E014C066ED76E08F
:1032A00011C062E976E00EC06DE776E00BC068E61B
:1032B00076E082EE95E00E94402B62E276E002C06A
:1032C0006CE076E082EE95E00E94402B6AE070E0D0
:1032D00080E090E00E94892982EE95E00E94662CB1
:1032E000892B29F082EE95E00E94932CF5CF08956A
:1032F000ACE1B0E0EEE7F9E10C94092F90914505BF
:103300009F3F09F023C1482F50E0FA013A97EF366A
:10331000F10508F00FC1E15CFF4F0C94362F61E11D
:1033200072E0A0C06DE172E082EE95E00E94522B47
:1033300085E789838BE1EFE9F5E0DE0112960190E4
:103340000D928A95E1F76CE1CE0101960E940D0C79
:103350000E948B0B83E08093730568EC70E080E043
:1033600090E00E94892980917305843009F0E2C0C1
:103370008FE70E94A9090E94BC098983853509F05D
:10338000D9C06DEE74E082EE95E00E94402B6FECA8
:1033900074E082EE95E00E94402B61EB74E096C0F1
:1033A00065E372E082EE95E00E94522B89E6898304
:1033B00061E0CE0101960E940D0C0E948B0B83E010
:1033C0008093730568EC70E080E090E00E948929AA
:1033D00080917305843009F0ADC08FE70E94A90980
:1033E0000E94BC0989838E010E5F1F4F7E014DE153
:1033F000E40EF11C0E94BC09F80181938F01EE15C7
:10340000FF05C1F78BE1FE013296AFE9B5E001900F
:103410000D928A95E1F78981893409F08BC063E9BF
:1034200074E082EE95E00E94402B65E774E082EE46
:1034300095E00E94402B67E574E048C06FE472E0BD
:1034400082EE95E00E94522B8EEF8093450572C06C
:1034500080528750805390914805981708F066C0B5
:103460006EE572E082EE95E00E94522B63C084E12B
:103470008093450560E274E029C085E180934505AD
:1034800069EE73E023C086E18093450562EB73E04B
:103490001DC087E18093450568E673E017C088E1A9
:1034A0008093450567E573E011C089E18093450588
:1034B00063E473E00BC08AE1809345056EE273E03C
:1034C00005C08BE18093450566E073E082EE95E0F0
:1034D0000E94402B2FC06CEE72E082EE95E00E94BD
:1034E000402B8091AD0591E01DC066ED72E082EE4B
:1034F00095E00E94402B8091AD0592E013C061ECF5
:1035000072E082EE95E00E94402B8091AD0594E040
:1035100009C066EA72E082EE95E00E94402B80913D
:10352000AD0598E089278093AD058FEF8093450521
:103530000E94431082EE95E00E94662C892B09F4CC
:103540005BC182EE95E00E94932CF4CF0E94421161
:10355000882309F451C18091DF04811104C08FEFE9
:103560008093450541C140E050E060E070E080EEAE
:1035700094E00E94AD2F40914505042F112707FDCF
:103580001095212F312FF8013197EB31F10508F01B
:103590001BC1E255FF4F0C94362F552747FD509520
:1035A0002091480530E0241735070CF40DC18B013C
:1035B0009C01015011092109310900321105210531
:1035C000310558F0C0904905EBE4F5E0F12CD12C21
:1035D000A8E2EA2E415051090FC0FA01E156FA4F14
:1035E00061506083D9C0DF0111972C9130E024171E
:1035F000350729F0F3943296FC10F5CFCBC00E2D91
:1036000010E020E030E0061717072807390741F4DB
:103610002081DA01A156BA4F11962C93DD24D39460
:10362000E394E8CF6F3F71058105910511F008F033
:10363000CBC06093B705B0C06F3F710581059105A0
:1036400011F008F0C1C06093B805A6C06F3F7105C6
:103650008105910511F008F0B7C06093B9059CC0D1
:103660002091E00420622037E9F440E050E060E07F
:1036700070E081EE94E00E94AD2F9B01AC01DC0173
:10368000CB010197A109B1090897A105B10508F07F
:10369000AEC0A4EDB0E30E94872E6A5E7C4A8A46E3
:1036A000954E24C02636E9F440E050E060E070E03A
:1036B00081EE94E00E94AD2F9B01AC01DC01CB01B7
:1036C0000197A109B1090797A105B10508F08FC0BD
:1036D000A8EAB1E60E94872E645E7C438E46944E33
:1036E00005C0611571058105910579F08B019C017B
:1036F000005C1D49284535430130FAE51F07F2E615
:103700002F07F2E03F0708F05FC06093AF057093AA
:10371000B0058093B1059093B2053EC06F3F71052F
:103720008105910511F008F04FC06093B30534C0D6
:103730008B019C0101501109210931090F3F11052D
:103740002105310508F040C06093B40525C08B0108
:103750009C01045C1940210931090D344DE1140725
:103760002105310528F47093B6056093B50514C0A2
:10377000611571058105910521F48FEF8093AE05E8
:103780000BC06134710581059105F0F461506093BF
:10379000AE0502C0DD20C1F08091DE0481111AC0A7
:1037A00080917F0590918005A0918105B09182055F
:1037B0000196A11DB11D80937F0590938005A09374
:1037C0008105B093820506C060E772E082EE95E065
:1037D0000E94522B0E9438118FEF809345056AE0BA
:1037E00082EE95E00E94642B0E94431005C061E0C8
:1037F00070E080E090E07ACF6C96E8E00C94252FA2
:103800006AE572E082EE95E00E94402B62E472E08D
:1038100082EE95E00E94402B82EE95E00E94662C9D
:10382000892B31F082EE95E00E94932C0E9478194A
:103830000E945018823029F0833051F46DE072E01C
:1038400002C064E272E082EE95E00E94402B08958F
:103850008FEF809345051092DE040E944310809103
:1038600045058E3F69F082EE95E00E94662C892B1B
:10387000B1F382EE95E00E94932C0E947819EFCF6D
:1038800008950F931F93109145051F3F09F0D2C073
:10389000893409F457C000F5883309F469C058F435
:1038A000803309F477C008F061C08B3109F440C05F
:1038B0008132B1F1B9C0813409F487C030F4893361
:1038C00009F466C0803461F1AFC0823409F48EC05F
:1038D000863409F448C0A8C0823609F487C078F459
:1038E000883531F128F48235C1F18335E1F09CC08F
:1038F0008A3509F494C0813609F467C095C08237CF
:1039000061F128F4863679F18936E1F08DC0883787
:1039100079F08A3709F483C0833709F085C003C082
:1039200061E172E015C00E94730D6EE872E004C0A0
:103930000E947C0D68EA72E082EE95E00E94522BB4
:103940008EEF70C00E947A060E94BF0667EC72E09C
:1039500082EE95E00E94522B67C081E00E94DF0654
:1039600060EE72E0F5CF0E94ED105EC080535AC049
:103970006AEF71E082EE95E00E94402B90919E05E7
:1039800088E0890F8871977E892B80939E051AC0E5
:1039900089E048C067EE71E082EE95E00E94402B1E
:1039A0008091BF059091C005A091C105B091C2055D
:1039B00020E182278093BF059093C005A093C105A5
:1039C000B093C205109345052FC061ED71E082EE02
:1039D00095E00E94402B8091BF059091C005A09179
:1039E000C105B091C20540E4842710C060EC71E0CD
:1039F00082EE95E00E94402B8091BF059091C0051A
:103A0000A091C105B091C20520E282278093BF0535
:103A10009093C005A093C105B093C20502C00E9457
:103A2000001C8FEF80934505809145058E3F09F07E
:103A3000D4C0DDC00E944211882309F4D8C080910F
:103A4000DF04811104C08FEF80934505C6C040E0BC
:103A500050E060E070E080EE94E00E94AD2F0091B5
:103A60004505112707FD1095212F312FF8013197BA
:103A7000E930F10508F0B4C0E753FF4F0C94362F3E
:103A80008B019C01015C1D49284535430F3F1945B9
:103A90002246324008F0A4C060937B0570937C05F9
:103AA00080937D0590937E0577C060937F0570932A
:103AB0008005809381059093820581E08093DE04E8
:103AC0006BC0683071058105910508F089C060936D
:103AD000830562C08B019C01015011092109310944
:103AE0000A3011052105310508F07AC0609384057C
:103AF00053C061EB71E080EE94E00E94E73010E08B
:103B0000009799F00E94C130009779F0183130F495
:103B1000E12FF0E0EA58FA4F87871F5F61EB71E011
:103B200080E090E00E94E730EBCF1831A8F5E12F5C
:103B3000F0E0EA58FA4F17861F5FF7CF653071053E
:103B40008105910508F04CC060939D0525C08B014F
:103B50009C01015011092109310906301105210587
:103B60003105F0F520919E05287F262B20939E0598
:103B700013C08B019C010150110921093109011564
:103B8000124C2140310560F56093770570937805FC
:103B90008093790590937A058091DE04811113C09A
:103BA00080917F0590918005A0918105B09182055B
:103BB0000196A11DB11D80937F0590938005A09370
:103BC0008105B09382050E9438118FEF80934505DF
:103BD0006AE082EE95E00E94642B0E94F31807C011
:103BE00060E772E082EE95E00E94522BECCF1F91CD
:103BF0000F9108958FEF809345051092DE040E9487
:103C0000F318809145058E3F69F082EE95E00E94A1
:103C1000662C892BB1F382EE95E00E94932C0E94D2
:103C2000411CEFCF6AE070E080E090E00E948929BB
:103C300082EE95E00E94662C892B29F082EE95E0B9
:103C40000E94932CF5CF0895CF93C82F682F82EE52
:103C500095E00E94C02C90916A059C2790936A057C
:103C6000CF910895A1E0B0E0E8E3FEE10C940F2FBE
:103C700099830E94241E9981892F0E94241E2196D7
:103C8000E2E00C942B2F1F93CF93DF93182FEB01BF
:103C900010926A0565EB70E082EE95E00E9459068D
:103CA00062E670E082EE95E00E945906812F0E9444
:103CB000241ECE010E94321EDF91CF911F910895E4
:103CC00060916A0582EE95E00E94C02C0895A1E201
:103CD000B0E0EDE6FEE10C940B2F7B018A018C3005
:103CE00009F453C108F040C0863009F4BCC018F58F
:103CF000833009F491C070F4813009F472C08230CD
:103D000009F048C26BE170E082E00E94431E0FE9B7
:103D100015E078C0843009F487C0853009F03AC2D4
:103D20006091490570E0660F771F85E00E94431E91
:103D30000AE415E086C0893009F4A7C070F4873022
:103D400009F49BC0883009F025C261E070E088E08A
:103D50000E94431E8091D40523C28A3009F4CAC050
:103D60008B3009F4F2C016C28A3609F475C1D8F452
:103D7000873609F43AC138F4853609F40EC186361F
:103D800009F41FC107C2883609F437C1893609F022
:103D900001C261E070E089E60E94431E0E947A063B
:103DA0000E94BF06F5C18D3609F4D4C138F48B36B4
:103DB00009F491C18C3609F49AC1ECC18E3609F42C
:103DC000DCC1873C09F0E6C161E070E087EC0E944D
:103DD000431E81E00E94241E0E94601E10926B050B
:103DE000E3C169E270E081E00E94431E06E715E04E
:103DF000F80181918F010E94241EF5E00F391F0701
:103E0000B9F7D0C1F80181918F010E94241EF5E01D
:103E10000A3B1F07B9F7C6C161E070E083E00E946A
:103E2000431E0E945018BCC161E070E084E00E9413
:103E3000431E81E00E94241E0E94601E0E94831681
:103E4000B3C18091490590E0880F991F98012A54C9
:103E500035402817390708F0A5C1F80181918F0175
:103E60000E94241EEECF62E070E086E00E94431EB6
:103E700084E893E00E94321E95C161E070E087E023
:103E80000E94431E809148058BC186E6898361E0CC
:103E9000CE0101960E940D0C0E948B0B83E0809353
:103EA000730568EC70E080E090E00E9489298091C1
:103EB00073058430D9F48FE70E94A9090E94BC09D8
:103EC0008983863469F460E270E089E00E94431ED1
:103ED00010E20E94BC090E94241E1150D1F762C159
:103EE00061E070E089E00E94431E52C161E070E031
:103EF00089E053C169E170E08AE00E94431E82E0DC
:103F00008093BA05209172058091BF059091C005FC
:103F1000A091C105B091C205222311F0806801C0B3
:103F20008F778093BF059093C005A093C105B09390
:103F3000C2050AEB15E0F80181918F010E94241E51
:103F4000F5E0033D1F07B9F72DC161E270E08BE09A
:103F50000E94431E8091AA048F3F39F08091AA04E9
:103F600091E0980F9093AA0402C08091AA040E9445
:103F7000241E10E0812F0E9410160E943C090E940E
:103F8000321E1F5F1031B1F70DC161E070E08CE0AF
:103F90000E94431E8091D30503C161E070E085E675
:103FA0000E94431E89E2E816F10409F0F8C0D80126
:103FB000E6E7F5E08D91819385E0EF39F807D1F7D9
:103FC000E7C061E070E086E60E94431EEBE1EE167A
:103FD000F10409F0E4C0D801EFE9F5E08D91819397
:103FE00085E0EA3BF807D1F7D3C061E070E087E6EF
:103FF0000E94431E0E94730DCBC061E070E088E612
:104000000E94431E85E789838BE1EFE9F5E0DE013D
:10401000129601900D928A95E1F76CE1CE0101961E
:104020000E940D0C0E948B0B83E08093730560E26D
:1040300073E080E090E00E948929809173058430CC
:1040400009F0ADC08FE70E94A9090E94BC098983CD
:10405000853509F0A4C09CC061E070E08AE60E944A
:10406000431E89E6898361E0CE0101960E940D0C12
:104070000E948B0B83E08093730560E273E080E025
:1040800090E00E94892980917305843009F087C0EF
:104090008FE70E94A9090E94BC0989838E010E5FE7
:1040A0001F4F7E01EDE1EE0EF11C0E94BC09F801EC
:1040B00081938F01EE15FF05C1F78BE1FE0132966A
:1040C000AFE9B5E001900D928A95E1F789818934D5
:1040D00009F065C05DC061E070E08BE60E94431EA0
:1040E000F80180818093D4050E947C0D51C061E06D
:1040F00070E08CE60E94431EF0E2EF16F10461F4DA
:1041000087E6898380E2F801DE01129601900D9224
:104110008A95E1F761E203C087E4898361E0CE011B
:1041200001960E940D0C0E948B0B83E08093730517
:104130006CE474E080E090E00E948929809173052E
:10414000843069F58FE70E94A9090E94BC09873471
:1041500031F51EC061E070E08DE60E94431E89E1EA
:10416000E816F104E1F4D801EAEBF5E08D918193D2
:1041700085E0E33DF807D1F70BC061E070E08EE623
:104180000E94431EF80180818093D3050E945D0D3B
:1041900081E006C061E070E08AEC0E94431E80E08E
:1041A0000E94241E0E94601EA196E6E00C94272F18
:1041B000A0E0B0E0EEEDF0E20C94092FCAECD3E001
:1041C00014E606E035E0F32E44E0E42E53E0D52E6D
:1041D00062E0C62E82EE95E00E94662C892B09F4DF
:1041E0009BC082EE95E00E94932C282F809335048B
:1041F0004091340450E04730510560F7FA01EE5227
:10420000FF4F0C94362F853B29F781E080933404CF
:10421000E1CF823609F07DC0C0923404DBCF8093B9
:10422000330480933204D0923404D4CF9C013327DA
:104230003093310420933004909132049827909366
:104240003204E0923404C6CF382F22274091300444
:1042500050913104242B352B3093310420933004BA
:1042600090913204982790933204F09234042536CA
:10427000310508F4AFCF61E070E08CEC0E94431E82
:1042800081E00E94241E0E94601E43C020912E04E3
:1042900030912F04F901E653FC4F80839091320452
:1042A000982790933204C901019690932F0480932C
:1042B0002E0420913004309131048217930708F4C2
:1042C00089CF0093340486CF8091320482130BC0CF
:1042D00060912E0470912F044AEC53E080913304D6
:1042E0000E94671E0DC062E070E08BEC0E94431ECE
:1042F000809133040E94241E80916A050E94241E2E
:10430000FE01812F11928A95E9F710922F041092E5
:104310002E04109234045ECFCDB7DEB7E8E00C94E3
:10432000252F81E080936B0580916B05882349F0F0
:1043300082EE95E00E94662C892BB1F30E94D82072
:10434000F3CF0895AAE2B0E0E8EAF1E20C94072F77
:104350000E945A296B017C0181E00E94B00A82EE22
:1043600095E00E94662C892B29F082EE95E00E9450
:10437000932CF5CF4398299811E072E6B72EE9E225
:10438000AE2E03E00E945A296C197D098E099F09FF
:10439000693C710581059105F0F11123E1F10E945D
:1043A0005A296B017C0185B1846285B980ED97E063
:1043B0000E94B607B982E6E7F5E0DE0112968A2D83
:1043C00001900D928A95E1F76AE2CE0101960E9472
:1043D0000D0C85B18B7D85B980E090E00E94B60719
:1043E000009373050E948B0B62E370E080E090E025
:1043F0000E94892980917305843061F400937305CC
:104400008FE70E94A9090E94BC0911E0823419F4C7
:1044100010E001C011E087E00E947F2A892BB1F4EF
:1044200011E014C0439A299A85B1846285B982EE5D
:1044300095E00E94932C8D309105C1F074F40A9799
:10444000A9F04398299885B18B7D85B982EE95E0D6
:104450000E94662C892B31F795CF8332910579F034
:104460008234910571F70E949121EBCF62EB71E0EC
:1044700082EE95E00E94402B0E94FA1DE2CF0E943E
:104480008316DFCF8F929F92AF92BF92CF92DF922F
:10449000EF92FF921F93CF93DF9387E00E947F2AD2
:1044A000892B09F089C068EC70E080E090E00E9400
:1044B000892980E090E00E94B6070E945A294B01AA
:1044C0005C016B017C0180ECC80E82E1D81EE11C0E
:1044D000F11C0E945A296C157D058E059F0530F44C
:1044E00087E00E947F2A892BA1F364C087E00E94A5
:1044F0007F2A892B09F05EC080ED97E00E94B60705
:104500000E945A296B017C01D0E0C1E088E4880E4A
:1045100086E2981EA11CB11C11E087E00E947F2A50
:10452000892B21F58C149D04AE04BF0430F480ED7A
:1045300097E00E94B607D1E0F0CF0E945A296C198B
:104540007D098E099F09693C71058105910528F354
:104550000E945A296B017C01C12719F080ED97E078
:1045600002C080E090E00E94B607D7CF80E090E0E4
:104570000E94B607DD23B9F08091D30590E0019643
:1045800065E070E00E94AA2E8093D3050E945D0D25
:104590000E94DC130E947C0D64EF71E080E090E0EB
:1045A0000E94892909C080E00E94DF060E94F41160
:1045B0000E94730D0E94A221DF91CF911F91FF9065
:1045C000EF90DF90CF90BF90AF909F908F90089525
:1045D000CF92DF92EF92FF9280E00E940D080E943E
:1045E000E40761E081E10E94132A61E08DE00E940E
:1045F000132A61E089E00E94132A61E08AE00E94A8
:10460000132A60E087E00E94132A60E08BE00E949A
:10461000132A61E08BE00E944C2A60E08CE00E944B
:10462000132A61E08CE00E944C2A60E088E00E943E
:10463000132A61E088E00E944C2A0E949F0740E014
:1046400052EC61E070E082EE95E00E94AE2D0E9497
:10465000DC130E947C0D0E94C1138FEF8093AA048B
:104660000E94F90778940E945A296B017C0180917D
:10467000AA048F3F59F40E945A296C197D098E09AA
:104680009F09603D77408105910588F380ED97E0B3
:104690000E94B60761E087E00E944C2A439A299A5B
:1046A00082EE95E00E94662C892B29F082EE95E03F
:1046B0000E94932CF5CF6DEF72E082EE95E00E94A0
:1046C000212B84E893E00E94620C64E173E082EEA7
:1046D00095E00E94212B4AE050E063E070E082EE1A
:1046E00095E00E94F12B62E370E080E090E00E9490
:1046F000892982EE95E00E94662C04970CF182EEE7
:1047000095E00E94932C82349105D1F482EE95E0DD
:104710000E94932C8E34910599F482EE95E00E94CC
:10472000932C8434910561F482EE95E00E94932CE1
:10473000819731F480E090E00E94B6070E94A221A8
:1047400040917705509178056091790570917A05CF
:10475000DB01CA010197A109B1090497A105B105BF
:1047600068F44093A904433029F440EA56E861E034
:1047700070E004C040E052EC61E070E082EE95E051
:104780000E94AE2D0E9442224398299880E090E03A
:104790000E94B6070E94C1131092C5048091BF0504
:1047A00083FF11C080918B05882351F08091920581
:1047B000882331F080919905882311F087E001C0AA
:1047C00085E08093C50480E00E94B00A8091C60411
:1047D0000E94E4090E948B0B10923F0410923E0449
:1047E00010923D04F12C8091D4058F15B0F062E356
:1047F00070E080E090E00E94892980ED97E00E94BF
:10480000B60762E370E080E090E00E94892980E0D2
:1048100090E00E94B607F394E6CF80919E0584FF56
:1048200008C0982F987181E0983109F080E00E94CB
:10483000B0118FE00E940D08FF90EF90DF90CF90B5
:104840000895EF92FF920F931F93CF93DF938C0104
:104850006EE770E082EE95E00E945906E801F12CC7
:10486000F0E2EF2E8E0188818D57823048F46DE79B
:1048700070E082EE95E00E94590688818E2588833B
:104880002196F801608182EE95E00E94C02CF3949D
:10489000F9E0FF12E7CF6EE770E082EE95E00E944C
:1048A0005906CDB7DEB7E6E00C94272FA9E0B0E0BB
:1048B000ECE5F4E20C940F2F9091C70491110EC017
:1048C0009EEF99838A836B8350E0559547954C837F
:1048D0002D83198618861F821E822EC04091CC041B
:1048E000842F90E0B4E095958795BA95E1F7242F51
:1048F0002F7030E08217930719F18DEF89831B82A7
:10490000FE01349650E0842F90E0A4E095958795C1
:10491000AA95E1F7242F2F7030E08217930749F012
:10492000DC01A353BB4F8C918193405F5F5F563096
:1049300051F74093CC045A83CE0101960E94212462
:104940008091C70490E0019666E070E00E94AA2E74
:104950008093C7042996E2E00C942B2FA0E0B0E0EE
:10496000E4EBF4E20C94082F6C016EE770E082EE49
:1049700095E00E9459068601E12CF12CC0E0D0E0C0
:1049800030E2B32EF801608183E8860F823078F43C
:104990006DE770E082EE95E00E945906F8016081B3
:1049A0006B2570E082EE95E00E94590604C082EE0D
:1049B00095E00E94C02CE114F10459F0F8018081C7
:1049C0009E01280F311DC901C92FDD27C80FD91F2E
:1049D000DD273FEFE31AF30A89E0E816F10459F006
:1049E00028E0E216F10421F48C2F8095F6018087EF
:1049F0000F5F1F4FC7CFCDB7DEB7E9E00C94242F70
:104A0000A9E0B0E0E6E0F5E20C940F2FE82F362F96
:104A10008091C70490E0019664E270E00E94AA2EA3
:104A20008093C70458E9598350E15A83813089F053
:104A300048F08230B9F08330D9F48B8381EF8C83D6
:104A40003D8319C085E08B8381EF8C832F5F2D839D
:104A500012C08B8381EF8C8384E6489FA0011124D0
:104A60005D8309C084E08B8381EF8C83ED8303C079
:104A70000E94ED1104C0CE0101960E94AE24299639
:104A8000E2E00C942B2FA2E0B0E0E9E4F5E20C9414
:104A9000042F182F762E2A8349830E9466296B01E2
:104AA0007C018091DD048090C8049090C904A0909E
:104AB000CA04B090CB042A8149818823C1F0D70170
:104AC000C60188199909AA09BB094C015D0191EE3B
:104AD00089169EE29906A104B10420F1241708F476
:104AE000422F202F672D812F0E94002513C0D70150
:104AF000C60188199909AA09BB094C015D0191E316
:104B0000891695E79906A104B10460F0672D812FFD
:104B10000E945624C092C804D092C904E092CA04EC
:104B2000F092CB042296EDE00C94202FA2E2B0E0AC
:104B3000ECE9F5E20C94052F8CE00E94CB09811181
:104B40000FC06CE173E082EE95E00E94522B439A15
:104B5000299A80E00E94B00A0E948B0B4398299802
:104B600082EE95E00E94662C892B01F182EE95E0A1
:104B70000E94932C9091A904992319F00E94181473
:104B8000EFCF40913E0450E09A012F5F3F4F2F71CD
:104B9000332760913F0470E02617370709F3FA01C5
:104BA000E75BFB4F808320933E04DACF809173054F
:104BB000843009F086C00E9466296115710581055F
:104BC000910549F06093B7047093B8048093B904D9
:104BD0009093BA040CC081E090E0A0E0B0E0809334
:104BE000B7049093B804A093B904B093BA04809129
:104BF000AD049091AE0481609093AE048093AD04B7
:104C000083E0809373058FE70E94A90909E614E009
:104C10000E94BC09F80181938F01F4E002371F075D
:104C2000B9F72091720480916904982F922796FF1A
:104C30003BC090E4922790937204982F9873983316
:104C4000F1F410E0212F30E080916904877090E04A
:104C5000821793074CF11F5F20919E05812F90E0F2
:104C6000FC01E759FB4F24FF04C080810E94CF1153
:104C7000E9CF608182EE95E00E94C02CE3CF8F7374
:104C800099F480916A048093B60480916B048093B8
:104C9000B40480916C048093B30480916F0490E01D
:104CA0009093AC048093AB0480913D04813019F45F
:104CB00082E080933D0480913D04833011F4109292
:104CC0003D040E9466296B017C018091AF049091A4
:104CD000B004A091B104B091B2040097A105B10550
:104CE000C9F0A7019601281B390B4A0B5B0BDA01AF
:104CF000C901883B9B40A105B10560F00E94FA09FB
:104D00008093B5041092AF041092B0041092B104D5
:104D10001092B2048091BB049091BC04A091BD0498
:104D2000B091BE0446015701881A990AAA0ABB0A23
:104D300086E795E00E94270886169706A806B9061A
:104D400008F4B3C0C092BB04D092BC04E092BD048E
:104D5000F092BE040E9457068091AA048830A0F009
:104D60008091BF059091C005A091C105B091C20589
:104D70005CE1B695A795979587955A95D1F7892BBC
:104D80008A2B8B2B09F0C0C18091AA048F5F80937E
:104D9000AA048091B7049091B804A091B904B0918D
:104DA000BA040097A105B105F1F0C81AD90AEA0AB8
:104DB000FB0A86E795E00E9427086C157D058E05A5
:104DC0009F0508F013C18091BF0584FD04C080EDEC
:104DD00097E00E94B6071092B7041092B8041092A0
:104DE000B9041092BA0490917204907C909372046A
:104DF00050913E0480913F0420913D04581709F4DE
:104E000012C1223009F00FC1905890937204E091C2
:104E10009E05E770F0E0E658FC4F6081693008F0CD
:104E2000EAC0615040E04613E8C080933F0487E346
:104E3000840F90917204892B8093720440934004F4
:104E400083E080933D0485B1846285B91091830528
:104E50008091C504811136C18091BF0582FD3EC19C
:104E6000812F0E94AB0A8091C6040E94E409E09160
:104E70009E05E770F0E0E658FC4F608182E794E021
:104E80000E94C60B8091BF0582FD32C1E091C6042D
:104E9000EF5FE093C604E83109F433C1F0E0EA586B
:104EA000FA4F8785882309F42CC10E94350C813084
:104EB00069F580919E05887149F18091AD049091CA
:104EC000AE04880F991F9093AE048093AD0483E0E5
:104ED000809373050E948B0B0E9466296093AF0438
:104EE0007093B0048093B1049093B204672B682B45
:104EF000692B61F481E090E0A0E0B0E08093AF0422
:104F00009093B004A093B104B093B20480919E0535
:104F100084FF1FC08091AD049091AE048E7F0E94EB
:104F20005D09182F6091AB048091B6040E940E14A5
:104F3000482F612F8091B50449A30E940E1400915F
:104F4000D405282F49A16091B3048091B4040E9434
:104F5000432585B18B7D85B98091C3048130C1F033
:104F600018F08230B1F1DEC087E00E947F2A892BE1
:104F700009F0D8C081E08093C3040E945A2960934D
:104F8000BF047093C0048093C1049093C204CAC04C
:104F900087E00E947F2A892B31F50E945A29C09010
:104FA000BF04D090C004E090C104F090C2046C191A
:104FB0007D098E099F09693E73408105910508F4BA
:104FC000B1C082E08093C30480ED97E00E94B607F1
:104FD000A9C087E00E947F2A892B09F4A3C080E042
:104FE00090E00E94B6071092C3049CC080E090E05D
:104FF0000E94B607F8CE68E015CF851709F415CFE3
:105000004F5F242F30E090E0F901EE58FB4FDC01B8
:10501000A75BBB4F7C917083F901E05CFB4F708311
:1050200001968F7100CF2430B1F42091400481E4C7
:1050300094E0A3E7B4E0FC013E2F381B321718F4CC
:1050400031913D93F9CF87E3820F90917204892BC0
:1050500080937204F5CE8091C304823059F491603C
:1050600090937204439A299A8E010F5F1F4FF12C7F
:10507000B80111C04398299880913D04811103C063
:1050800081E080933D0480913D04833069F784E0A2
:1050900080933D04E9CF8F2D69A37AA30E94101657
:1050A000F801819391938F01F39469A17AA1F0E1C2
:1050B000FF12F1CF80919E0543E754E087700E9474
:1050C000AC08C1CE112309F4C7CE9091C40421E0ED
:1050D000290F2093C4049813BFCE20C08BE00E94F8
:1050E0007F2A892B09F0BCCE439A299A17E0B8CEC3
:1050F0008BE00E947F2A892B09F0C8CE439829981B
:10510000C5CE1092C604D1CE8091AA04883011F485
:10511000439A299A89E08093AA04C7CE1092C404C6
:1051200011509ACEA296ECE00C94212F8230E8F434
:10513000E82FF0E0EE0FFF1FEB52FA4F7183608310
:10514000813041F0809169008C7F842B80936900CD
:10515000E89A089580916900440F551F440F551F28
:10516000837F842B80936900E99A08951F920F92A0
:105170000FB60F9211242F933F934F935F936F932A
:105180007F938F939F93AF93BF93EF93FF93809100
:10519000D5059091D605892B29F0E091D505F091A0
:1051A000D6050995FF91EF91BF91AF919F918F9196
:1051B0007F916F915F914F913F912F910F900FBE13
:1051C0000F901F9018951F920F920FB60F921124F7
:1051D0002F933F934F935F936F937F938F939F93FF
:1051E000AF93BF93EF93FF938091D7059091D8052C
:1051F000892B29F0E091D705F091D8050995FF9109
:10520000EF91BF91AF919F918F917F916F915F913E
:105210004F913F912F910F900FBE0F901F901895B7
:105220001F920F920FB60F9211242F933F938F93DB
:105230009F93AF93BF938091DA059091DB05A09186
:10524000DC05B091DD053091D90523E0230F2D3722
:1052500020F40196A11DB11D05C026E8230F02967A
:10526000A11DB11D2093D9058093DA059093DB052C
:10527000A093DC05B093DD058091DE059091DF05FC
:10528000A091E005B091E1050196A11DB11D8093AB
:10529000DE059093DF05A093E005B093E105BF9193
:1052A000AF919F918F913F912F910F900FBE0F90D3
:1052B0001F9018952FB7F8946091DA057091DB056F
:1052C0008091DC059091DD052FBF08953FB7F894DC
:1052D0008091DE059091DF05A091E005B091E10598
:1052E00026B5A89B05C02F3F19F00196A11DB11D41
:1052F0003FBF6627782F892F9A2F620F711D811D5E
:10530000911D42E0660F771F881F991F4A95D1F7BC
:105310000895CF92DF92EF92FF92CF93DF936B01CC
:105320007C010E946629EB01C114D104E104F1045F
:1053300079F00E9466296C1B7D0B683E7340A0F3D8
:1053400081E0C81AD108E108F108C851DC4FECCF60
:10535000DF91CF91FF90EF90DF90CF9008957894F8
:1053600084B5826084BD84B5816084BD85B582606A
:1053700085BD85B5816085BDEEE6F0E08081816008
:105380008083E1E8F0E01082808182608083808108
:1053900081608083E0E8F0E0808181608083E1EBE0
:1053A000F0E0808184608083E0EBF0E080818160C8
:1053B0008083EAE7F0E0808184608083808182607E
:1053C0008083808181608083808180688083109267
:1053D000C1000895833081F028F4813099F0823043
:1053E000A1F008958630A9F08730B9F08430D1F467
:1053F000809180008F7D03C0809180008F778093A3
:105400008000089584B58F7702C084B58F7D84BDF8
:1054100008958091B0008F7703C08091B0008F7D98
:105420008093B0000895CF93DF9390E0FC01ED509E
:10543000F44F2491FC01E95FF34F8491882349F1F3
:1054400090E0880F991FFC01E15DF34FA591B491A5
:105450008B5D934FFC01C591D4919FB7611108C03A
:10546000F8948C91209582238C93888182230AC0A2
:10547000623051F4F8948C91322F309583238C93C1
:105480008881822B888304C0F8948C91822B8C9322
:105490009FBFDF91CF910895A1E0B0E0E2E5FAE28D
:1054A0000C940D2F282F30E0F901E152F44F849134
:1054B000F901ED50F44F1491F901E95FF34F0491B4
:1054C0000023C9F0882321F069830E94EA296981B9
:1054D000E02FF0E0EE0FFF1FEB5DF34FA591B491CD
:1054E0009FB7F8948C91611103C01095812301C07E
:1054F000812B8C939FBF2196E4E00C94292FCF93AE
:10550000DF93282F30E0F901E152F44F8491F90143
:10551000ED50F44FD491F901E95FF34FC491CC23DE
:1055200091F081110E94EA29EC2FF0E0EE0FFF1FAD
:10553000E55EF34FA591B4912C912D2381E090E08D
:1055400021F480E002C080E090E0DF91CF910895E7
:105550008E3008F08E50877020919D0190E4299F35
:1055600090011124822B80937C0080917A008064CA
:1055700080937A0080917A0086FDFCCF809178003C
:105580002091790090E0922B0895A0E0B0E0EBEC40
:10559000FAE20C94092F6C017A01EB01E60EF71E7A
:1055A00000E010E0CE15DF0561F06991D601ED91C4
:1055B000FC910190F081E02DC6010995080F191F9B
:1055C000F1CFC801CDB7DEB7E8E00C94252F611507
:1055D000710589F0DB010D900020E9F7AD01415024
:1055E0005109461B570BDC01ED91FC910280F381C0
:1055F000E02D0995089580E090E00895EF92FF92E4
:105600000F931F93CF93DF938C01FB01C0E0D0E099
:1056100064917F018FEFE81AF80A662361F0D801E0
:10562000ED91FC910190F081E02DC8010995C80F22
:10563000D91FF701EDCFCE01CDB7DEB7E6E00C9470
:10564000272F0E94E72A0895DC01ED91FC9101903B
:10565000F081E02D099508950F931F93CF93DF9369
:10566000EC016DE00E94242B8C016AE0CE010E94C7
:10567000242B800F911FDF91CF911F910F910895DF
:105680000F931F93CF93DF93EC010E94FE2A8C01AE
:10569000CE010E942C2B800F911FDF91CF911F9183
:1056A0000F9108950F931F93CF93DF93EC010E9406
:1056B000E72A8C01CE010E942C2B800F911FDF91D5
:1056C000CF911F910F9108950F931F93CF93DF9365
:1056D000EC010E94242B8C01CE010E942C2B800F08
:1056E000911FDF91CF911F910F910895A1E2B0E03A
:1056F000ECE7FBE20C94052F7C01C42EE52FCB01D7
:10570000D22E19A221E02D1510F02AE0D22E8E0102
:105710000F5D1F4F8D2C912CA12CB12C6C2D7E2F49
:10572000A50194010E94BE2E8C2DD29E80191124B9
:10573000015011098A3010F4805D01C0895CF801C4
:105740008083211531054105510521F0C22EE32F3B
:10575000CA01E4CFB801C7010E94E72AA196ECE094
:105760000C94212FA0E0B0E0E8EBFBE20C94092FB1
:10577000EC016A017B012115310541F4E881F981D1
:105780000190F081E02D642F09951DC02A3031056C
:10579000A9F477FF12C06DE20E94242B8C014427EC
:1057A0005527BA014C195D096E097F092AE0CE011F
:1057B0000E94762B800F911F06C02AE0B701A60138
:1057C000CE010E94762BCDB7DEB7E8E00C94252FF2
:1057D0009A01AB01662757FD6095762F0E94B22B88
:1057E00008950F931F93CF93DF93EC019A01AB01C0
:1057F000662757FD6095762F0E94B22B8C01CE0153
:105800000E942C2B800F911FDF91CF911F910F9140
:1058100008952115310549F4DC01ED91FC910190C9
:10582000F081E02D642F099508950E94762B08954C
:105830009A01462F50E060E070E00E94092C089524
:105840009A01AB0160E070E00E94092C08950F936B
:105850001F93CF93DF93EC010E94092C8C01CE01A2
:105860000E942C2B800F911FDF91CF911F910F91E0
:1058700008950F931F93CF93DF93EC019A01AB012F
:1058800060E070E00E94092C8C01CE010E942C2B5C
:10589000800F911FDF91CF911F910F9108950F936A
:1058A0001F93CF93DF93EC019A01462F50E060E005
:1058B00070E00E94092C8C01CE010E942C2B800FDD
:1058C000911FDF91CF911F910F910895FC012485C5
:1058D0003585F901E05CFF4F80819181F901EE5B34
:1058E000FF4F20813181821B930B8F73992708957D
:1058F000FC0184859585FC01E05CFF4F408151816E
:10590000FC01EE5BFF4F208131814217530741F0CC
:105910000190F081E02DE80FF91F808190E008955B
:105920008FEF9FEF0895FC0184859585FC01E05C75
:10593000FF4F40815181FC01EE5BFF4F208131819F
:105940004217530779F0A081B181A80FB91F8C913C
:10595000208131812F5F3F4F2F7333273183208385
:1059600090E008958FEF9FEF0895FC0181A18823B7
:1059700029F0A489B5898C9186FFFBCF11A20895E7
:10598000CF93DF93FC0126853785D901A05CBF4FFB
:105990008D919C91119701968F739927E901CE5BA8
:1059A000DF4F4881598184179507D9F30D90BC9139
:1059B000A02DA20FB31F6C93A685B785A05CBF4F27
:1059C00011969C938E93A689B7892C9181E090E0E3
:1059D000078C02C0880F991F0A94E2F7282B2C939A
:1059E00081E081A30488F589E02D80818064808333
:1059F00081E090E0DF91CF91089508951F920F927A
:105A00000FB60F9211242F933F934F938F939F9331
:105A1000EF93FF938091C00082FD1CC04091C600AF
:105A2000809188069091890601968F73992720911D
:105A30008A0630918B068217930771F0E0918806F1
:105A4000F0918906E85BF94F408390938906809333
:105A5000880602C08091C600FF91EF919F918F91BF
:105A60004F913F912F910F900FBE0F901F9018955F
:105A700082EE95E00E94662C892B11F00E94FD2C8D
:105A800008951F920F920FB60F9211242F933F93F8
:105A90008F939F93EF93FF93209144063091450697
:105AA00080914606909147062817390731F4809176
:105AB000C1008F7D8093C10014C0E0914606F09133
:105AC0004706EC5FF94F208180914606909147068A
:105AD00001968F73992790934706809346062093EB
:105AE000C600FF91EF919F918F913F912F910F9061
:105AF0000FBE0F901F901895A0E0B0E0E2E8FDE225
:105B00000C94052FFC011382128288EE93E0A0E032
:105B1000B0E084839583A683B7838CEB93E0918375
:105B200080837587648757874687318B208B138BDB
:105B3000028BF58AE48AD78AC68AB18EA08E938EAC
:105B4000828E8F85848F8889858F8989868F8A89BF
:105B5000878F8B8980A3ECE00C94212FCF92DF926A
:105B6000EF92FF92CF93DF93EC016A017B01411525
:105B700081EE580761057105F9F0EC89FD8981E036
:105B800090E008A002C0880F991F0A94E2F7808372
:105B900060E079E08DE390E0A70196010E94BE2EBF
:105BA0002150310941095109569547953795279557
:105BB000211580E1380798F0EC89FD89108260E8B2
:105BC00074E88EE190E0A70196010E94BE2E21505C
:105BD0003109410951095695479537952795E88927
:105BE000F9893083EA89FB89208319A2EE89FF892C
:105BF000408181E090E09C010C8C02C0220F331F99
:105C00000A94E2F7422B4083EE89FF8940819C0190
:105C10000D8C02C0220F331F0A94E2F7422B4083FF
:105C2000EE89FF8940819C010E8C02C0220F331F38
:105C30000A94E2F7422B4083EE89FF8920810F8C82
:105C400002C0880F991F0A94E2F78095822380830F
:105C5000DF91CF91FF90EF90DF90CF9008958F92DA
:105C60009F92AF92BF92CF92DF92EF92FF920F93EB
:105C70001F9381E08F9385E08F9387E08F9383E07C
:105C80008F9384E08F93E6EC8E2E912CF2ECAF2E66
:105C9000B12CA1ECCA2ED12CB0ECEB2EF12C04ECE3
:105CA00010E025EC30E044E056E068E476E082EE77
:105CB00095E00E947C2D0F900F900F900F900F9009
:105CC0001F910F91FF90EF90DF90CF90BF90AF901A
:105CD0009F908F9008950E94AF290E94E822C8E308
:105CE000DDE20E9496252097E1F30E94382DF9CF3E
:105CF000A29FB001B39FC001A39F700D811D11240D
:105D0000911DB29F700D811D1124911D08950E9457
:105D1000782EA59F900DB49F900DA49F800D911D8E
:105D200011240895B7FF0C94872E0E94872E821BA2
:105D3000930B0895DB018F939F930E94872EBF9151
:105D4000AF91A29F800D911DA39F900DB29F900DCA
:105D50001124089597FB072E16F4009407D077FDC1
:105D600009D00E943C2F07FC05D03EF49095819508
:105D70009F4F0895709561957F4F0895A1E21A2E67
:105D8000AA1BBB1BFD010DC0AA1FBB1FEE1FFF1FDF
:105D9000A217B307E407F50720F0A21BB30BE40B2F
:105DA000F50B661F771F881F991F1A9469F7609576
:105DB0007095809590959B01AC01BD01CF01089530
:105DC000052E97FB1EF400940E94F72E57FD07D076
:105DD0000E94BE2E07FC03D04EF40C94F72E509573
:105DE0004095309521953F4F4F4F5F4F08959095C7
:105DF0008095709561957F4F8F4F9F4F08952F929B
:105E00003F924F925F926F927F928F929F92AF924A
:105E1000BF92CF92DF92EF92FF920F931F93CF9397
:105E2000DF93CDB7DEB7CA1BDB0B0FB6F894DEBF2E
:105E30000FBECDBF09942A88398848885F846E8454
:105E40007D848C849B84AA84B984C884DF80EE809E
:105E5000FD800C811B81AA81B981CE0FD11D0FB6A7
:105E6000F894DEBF0FBECDBFED010895EE0FFF1F0A
:105E70000590F491E02D0994AA1BBB1B51E107C0CA
:105E8000AA1FBB1FA617B70710F0A61BB70B881FCA
:105E9000991F5A95A9F780959095BC01CD01089559
:105EA0008F929F92AF92BF92CF92DF92EF92FF922A
:105EB000CF93DF93EC01688179818A819B816115A1
:105EC00071058105910521F464E279ED8BE597E098
:105ED0002DE133EF41E050E00E94E02E49015A01EC
:105EE0009B01AC01A7EAB1E40E94872E6B017C0103
:105EF000ACEEB4EFA50194010E94952EC60ED71EFC
:105F0000E81EF91EF7FE06C081E0C81AD108E108B4
:105F100080E8F80AC882D982EA82FB82C701B6010A
:105F20009F77DF91CF91FF90EF90DF90CF90BF9060
:105F3000AF909F908F9008950E94502F089586E013
:105F400091E00E94502F089560930601709307011D
:105F5000809308019093090108952F923F925F92D8
:105F60006F927F928F929F92AF92BF92CF92DF9269
:105F7000EF92FF920F931F93CF93DF938B01EA0170
:105F80006115710521F0DB018C9311969C9320978C
:105F900039F09E01225031092332310508F0D8C072
:105FA0007C016701BFEFCB1ADB0A5601F701608065
:105FB000862D90E00E94DF30892B11F07601F1CF21
:105FC000FDE26F120AC0570182E0A80EB11CD70192
:105FD00011966C90772473940BC0BBE26B1207C0D0
:105FE0005701E2E0AE0EB11CD70111966C90712CF6
:105FF000CE018F7E892B89F4B0E36B1237C0F50197
:1060000080818F7D8835D1F46180F2E0AF0EB11CC4
:10601000872D8260782EC0E1D0E0CA30D10551F1E1
:10602000C031D10521F0C830D10599F409C0CC2484
:10603000CA94DC2CEC2CAFE0FA2E22C0209769F732
:10604000C8E0D0E0CC24CA94DC2CEC2CFFE1FF2E7D
:1060500017C06FEF7FEFCB019E01442737FD4095BE
:10606000542F0E94BE2E69017A010AC02097A9F61A
:10607000CAE0D0E0E9E9CE2EDC2CEC2CE9E1FE2EE2
:10608000F50160E020E030E0A9014E01AA2497FC70
:10609000A094BA2C1F0170ED572E560CA9E0A5153F
:1060A00070F48FEB860D8A3118F499EC592E06C0E6
:1060B0008FE9860D8A3148F589EA582E560C852DD0
:1060C00090E08C179D070CF56F3FD9F0C216D306F0
:1060D000E406F50698F0C501B4010E949A2E9B01D2
:1060E000AC01852D90E0A0E0B0E0280F391F4A1FD9
:1060F0005B1F281739074A075B0710F46FEF01C0D1
:1061000061E03196D1016C90C5CF0115110551F0B8
:10611000662311F0319703C071FE04C03297D80195
:10612000ED93FC9370FE07C05095409530952195F6
:106130003F4F4F4F5F4F67FF10C082E290E0909358
:106140008D0680938C066FEF7FEF8FEF9FEF07C078
:1061500060E070E080E090E002C0B901CA01DF9128
:10616000CF911F910F91FF90EF90DF90CF90BF9054
:10617000AF909F908F907F906F905F903F902F9007
:106180000895FC0188279927E89421912032E9F3AA
:10619000293010F02E30C8F32B3241F02D3239F473
:1061A000689404C00E941331820F911D21912053E5
:1061B0002A30C0F31EF4909581959F4F0895911158
:1061C00050C0803219F089508550D0F7089548ECBE
:1061D00053E00E94EC300895FA01A191B08100973C
:1061E00019F41097E1F0CD01DC01CD010D900020F4
:1061F00011F4C00113C0FB012191222319F02015D5
:10620000D9F7F3CFFB012191201519F41E921196B5
:1062100006C02223C1F70D900020A1F7D001FA019A
:10622000A193B08308957AE0979F902D879F802D4A
:10623000910D11240895F999FECF92BD81BDF89A70
:10624000992780B50895262FF999FECF1FBA92BDE0
:1062500081BD20BD0FB6F894FA9AF99A0FBE019647
:0C6260000895992788270895F894FFCF2F
:10626C0000008E06200001000000FF00020002006A
:10627C000200020002000200020002000200020002
:10628C00020002000200020002000280250000054C
:10629C00400AA1204EA50020244EA52C2330C0126C
:1062AC0000001A400AA1204EA5001B1E27522C23C9
:1062BC00308025000005400AA1204EA50020244E68
:1062CC00A52C2330004B000006400AD0009D49004D
:1062DC007B289D492C233000E1000005400A450134
:1062EC00D7DC03B81E0EBF00232E48E801008A40FD
:1062FC000A6001555502AD1E20000023C8015458F8
:10630C002074696D656F75742100596573004E6F4B
:10631C00002C00386368004E2F41002C205B005D80
:10632C002028002900486F70206368616E6E656CD0
:10633C00200020402000456E746572696E672061F4
:10634C0064617074697665206368616E6E656C203B
:10635C0073656C656374696F6E2C207069636B690F
:10636C006E673A007363616E6E6572206D6F646563
:10637C00004E4F5420454E41424C45440053656EEF
:10638C0064696E672073657474696E677320746FCB
:10639C002052580A00526573657474696E672073D5
:1063AC00657474696E6773206F6E2052580A0041D1
:1063BC00626F727465642065646974730A00696E37
:1063CC0076616C69642073656C656374696F6E00CB
:1063DC000D0A496E76616C696420696E7075742063
:1063EC002D206469736361726465642107005365D1
:1063FC007474696E677320736176656420746F20A2
:10640C00454550524F4D0A0052657665727465646D
:10641C002073657474696E67732066726F6D2045A6
:10642C004550524F4D0A004C6F61646564206661A3
:10643C0063746F72792064656661756C74730A009D
:10644C004B657920616E64206368616E6E656C7358
:10645C002072616E646F6D697A65640A004F7065B5
:10646C006E4C52536E672054582073746172746969
:10647C006E672000206F6E20485720006D6F64758A
:10648C006C65206C6F636B65643F00342B34003893
:10649C0000382B340031320031322B3400313600CD
:1064AC0050504D0052535349005344410053434CF8
:1064BC0000525844005458440041494E004C424547
:1064CC0045500053504B54524D00534255530053BA
:1064DC00554D44004C4C494E440000070B0C101118
:1064EC001500B7012B032F033103350338033D038C
:1064FC00B7014003440349034D03510355035903AA
:10650C005D0363036A036F0374038D028D028D02B6
:10651C008D02160A1322312900000000C02CC52A56
:08652C00662C932C782CB52C91
:107E00000F92CDB7DEB7112484B714BE81FFF1D035
:107E100082E08093C00088E18093C10086E0809377
:107E2000C20080E18093C4008EE0CDD088249924E4
:107E3000CC24C394F5E0DF2EE1E1EE2E73E0F72EC3
:107E4000B6D0082F813479F4B2D08983C2D0898129
:107E5000823811F481E005C0813811F485E001C059
:107E600083E09ED09AC0823411F484E103C085344B
:107E700019F485E0B6D091C0853561F498D0082F0B
:107E800010E095D090E0982E8824802A912A880CC2
:107E9000991C82C0863521F484E0A3D080E0E1CF34
:107EA000843609F04CC083D082D0A82E80D0B82E62
:107EB00000E011E07CD0F80181938F01AE16D1F77C
:107EC00088D0FB2DF53489F4E0E0F1E00BC0F9999E
:107ED000FECF92BC81BC0894811C911C819180BD15
:107EE000FA9AF99AEA1598F358C08B2D863409F05E
:107EF00054C0F401F7BEE89507B600FCFDCFF401CD
:107F0000A0E0B1E02C9130E011968C91119790E0B7
:107F1000982F8827822B932B12960C01C7BEE895C9
:107F20001124329681E0A038B80761F7F401D7BE7A
:107F3000E89507B600FCFDCFE7BEE8952EC0843774
:107F4000F1F435D034D0182F32D0B82E42D0FB2DDA
:107F5000F63421F4F40105914F010CC0FB2DF534EA
:107F600049F4F999FECF92BC81BC0894811C911C04
:107F7000F89A00B5802F14D0115049F70EC08537FC
:107F800039F427D08EE10CD085E90AD08FE069CF93
:107F9000813511F488E017D01CD080E101D050CF9A
:107FA0009091C00095FFFCCF8093C600089580910A
:107FB000C00087FFFCCF8091C00084FD01C0A89560
:107FC0008091C6000895E0E6F0E098E19083808318
:107FD0000895EDDF803219F088E0F5DFFFCF84E10E
:107FE000DFCF1F93182FE3DF1150E9F7F2DF1F9166
:0E7FF0000895282E80E0E7DFEE27FF27099492
:027FFE0001057B
:0400000300007E007B
:00000001FF
